:020000041100E9
:10300000002373B52B4D2C4C28006361022601F080
:1030100069F94021FE2221742800284B009601F016
:10302000B3F9002836D1217CFF222800244B0096DA
:1030300001F0AAF900282DD1224BA2899A4226D16B
:10304000E389214A93420DD1204B6361204B2268D2
:10305000002A03D1002B01D043CB43C4280001F048
:103060007FF973BD1B4A934201D00023EFE71A4B4F
:103070001A4A1B68934206D9C02304222800217CE7
:103080009B0001F0F7F9114B6361154BDFE700235B
:103090002374EAE7CC233821AC2228009B01217459
:1030A00001F0E8F90028F2D10E4B63610E4BE38189
:1030B0000E4BCCE7643CFF1F085CFF1F145CFF1F36
:1030C000165CFF1F595900008305000011410011D3
:1030D000CCBC0011821500002C5CFF1F8713000080
:1030E000D8BC0011C9410011AAAAFFFFC0BC001141
:1030F000F7B5164B0192C318021D002000938823D8
:103100005B05D3181B685C1C1AD09CB2402C18D8E5
:103110008D781E0CAC466746CD782D023D43AE42FD
:1031200006D1019800280ED110000C70240A4C70B2
:1031300003249BB20733A343D218009B9A42DED3E9
:10314000FEBD4432F9E71000FAE7C046FC0F00006C
:10315000802213B503000324019189B25201073183
:103160009B18A14304305A1A88235B05C3181B68B7
:10317000591C03D190429241104016BD99B240298A
:1031800007D80B000733A343C0189042ECD30020AC
:10319000F3E74430F9E7134B134A1B68126810B584
:1031A000FA24934201D81A00F824104BE4021B6859
:1031B0009A4210D813000E4A12689A420ED3013375
:1031C00007D1F823DB029C4203D10A49054808F0E5
:1031D0000BFB200010BDFC24E402ECE7FE24E4021B
:1031E000F7E7C04600C0071100D0071100E0071143
:1031F00000F00711FFFFFF7FF0B59BB015000490B2
:103200000391402A00D9A0E006AB59801A80FFF74D
:10321000C2FF0400042816D9002206A9FFF768FFA0
:10322000052810D906AB1B88AB420CD1002D07D066
:10323000514B2A000499C01808F026FC002802D13E
:1032400001201BB0F0BD06AB1D8020000699FFF7E2
:103250007FFF041E7BD1069B0793FFF79CFF802313
:103260005B01C618802307001B039E4201D3F8268A
:10327000F60288235B05F31801931B68013302D023
:10328000019808F051FC3D49019808F0ADFA3B1D4A
:103290000293331D05938822029B52059B181B68DD
:1032A00008935A1C3CD044219AB20091402A04D879
:1032B0000320D11D814389B2009103991B0C8B42DD
:1032C00024D0402A22D80122300008A9FFF710FF9D
:1032D000021E1BD1380008A9FFF70AFF04000428CA
:1032E00031D9009A059B9B1880225201B218934253
:1032F00040D288235B05C118009A09A808F09CF900
:103300001D4B009A09A9F01808F03EFB009A029B99
:103310009446634402931A4B029AFB189A42BAD31A
:1033200088235B05FC1821680198013908F05CFAD4
:10333000200008F0F9FB039A07AB5A803000079988
:10334000FFF706FF0400002C03D1002079E70428D2
:10335000FBD988235B05E018069908F045FA03239A
:10336000EA1C9A4300D16BE7034B0499E01808F07C
:103370000BFB65E70424ECE704000011FFFFFF7F6F
:10338000F80F0000F7B505001400402A21D80027E7
:1033900001AE71803780FFF7FEFE042816D93A008F
:1033A0003100FFF7A5FE042810D93688BC420BD0A7
:1033B000BD4209D0221CB44200D9321C064B92B245
:1033C000C118280008F038F930B2FEBDC04300B281
:1033D000FBE703204042F8E70400001137B5042260
:1033E00004000D0001A81649FFF7CCFF02000428D5
:1033F0000BD1019BA34208D3AB4204D0104901A8D2
:103400000195FFF7F9FE01203EBD0E4C2368200018
:10341000019308F089FB019920000139019108F01E
:10342000E3F980235B01E418074B9C42EED10422B0
:10343000034901A80195FFF7DFFE0020E4E7C0463D
:103440005555000000C007110000081130B589B0C3
:1034500008F012FA10226946254808F0A5FB254B12
:10346000009A9A420ED1019B029A0F2B33D8002169
:1034700001240698013B08D2002900D00292029B49
:10348000013331D10023029325E0551CF2D1020013
:103490002100EFE710341022200004A908F084FB7B
:1034A000029B013301D1069B0293882304995B059B
:1034B000C918059B06981A03120B049105928142C4
:1034C00003D02B4201D108F0B7F8019B013B0193D7
:1034D000019B002BDED1029B002B03D004930498A8
:1034E0004168084709B030BDE025014C2D03EFE7E6
:1034F00000000111504859368022F8B5964C974B80
:10350000D200002120001C6008F086F92300944AB4
:1035100088331A60934B1A786A23002A00D011333B
:10352000E3620A232365904B37221B780821A363AB
:103530008E4B6018E361102323628D4B3B25636142
:10354000C823DB00A36123008C331A602823013ACF
:10355000E26321646364C267043A201DC2672000ED
:10356000BC3005602000C03001602000C430036022
:1035700020000635CC3005602000083DC8300560CD
:103580002000D03002602200D43211602200D832F4
:10359000136022000226E032200016604222DC3056
:1035A000026020001B3DE43005602000E83001602F
:1035B0002000EC30036023000520F4331860230062
:1035C000F0331A602300183290331A6023009433CA
:1035D000196023001E3A98331A60AF23DB00236082
:1035E000644BFA252363644B6448A3642300B93217
:1035F000FC33FF32AD00A260E56022611D60A06275
:103600007320E0656D386065A065FA2796203F015C
:103610008000E76465625960A0660920E0660020CA
:10362000616757496666E167564E57492667A06746
:103630000F601527676027001A219C373960270023
:103640000731A037396027004B49A837396021007E
:10365000F8310D6021006427A4310F6021005F3F25
:10366000AC310F602100033FB0310F602700B43749
:103670003D00C8272F6027003825B83738609D6087
:10368000424D96215D64424D8900DD61414D1962D4
:103690005D62F53DFF3D9D621E253949DD66596637
:1036A000996499673C49DE651E6618675867D96753
:1036B000BE233A495B00E1508130394BFF30235043
:1036C00004302150C42149006350C623E4205B002C
:1036D000E2500433E2503349334A344BD160344929
:1036E000800019503349E938FF3819503249043005
:1036F000195032493248D16132491163324951631C
:103700001900F4310860CE20304940001160304982
:10371000195019002F48F83108602F49D1658221CE
:103720002E4A89005A501A002D490832D1671A00D2
:103730002C49B432116088212B4A89005A501A0052
:103740002A49883211602A4ADA6407F0B5FF01205D
:1037500008F08AF8F8BDC0460004FF1FAC5EFF1FEA
:103760009069FF1F9C3EFF1F4A0AFF1F3A07000097
:1037700080C3C9019A02000050C300006A1800000B
:1037800088130000204E0000F009FF1F6509FF1F8D
:1037900068100000C4090000DC05000040420F0072
:1037A00010270000D91AFF1FFC00FF1F0000FF1F99
:1037B0008127FF1FC52AFF1F5D29FF1F251EFF1F31
:1037C0007523FF1F411EFF1FED1FFF1FB11DFF1FB0
:1037D0000124FF1FE924FF1FD918FF1FB923FF1F72
:1037E000C921FF1FD521FF1FB11CFF1F691DFF1F2E
:1037F0009D1CFF1F0223F0B501245E4D5E4E2B7011
:103800005E4B91B01C705E4F03933368002108201B
:10381000FB7006F0D9FD082006F0D0FC002398428A
:1038200005D0FA78552A02D0332A00D096E03360CA
:1038300008F09AF8FFF760FE1F2201240021514B87
:1038400010AE1A70504B1C70504B1970504B1968C9
:103850009143163A0A431A60602219689143403A2C
:103860000A431A6008F040F908F02EF8C120FF2141
:10387000484B80001A588A431A50C5229200985823
:103880008843BF39014399509858434908408021E3
:10389000C9010143802099509958C0050902090ABD
:1038A0000143995080213D48490107F03DFF032322
:1038B00022003B49019400933A4807F0CDFF2C22A7
:1038C000394905A807F0B8FE05AC617820780234C4
:1038D00006F094FCA642F8D1344C0020012106F0F9
:1038E000A1FD2268324B03201A40A023DB021343C0
:1038F0002360802322689B041343236022682D4B9E
:103900001A4080239B03134323602B4A2B4B934283
:1039100000D8012007F0E8FF07F0EEFF80232268BF
:10392000DB0413432360287807F06EFE039B1878AE
:10393000C0B207F0F1FF07F00FFF2149042008F0A3
:103940008BF806F087FE00F0A7F800F0E9FD00F024
:1039500091FE00F00BFA002011B0F0BD00932100A1
:10396000174A042007F0D0FF8023DB059C62FFF795
:103970006DFD5DE74A0AFF1F34F000409C3EFF1FCB
:10398000385CFF1F480AFF1F490AFF1F680AFF1F14
:10399000BCF0004000E100E0FF00FFFFA03EFF1F81
:1039A0002451FF1FA04EFF1FE8BB001114F0004080
:1039B000FF7FF8FFFFFF9FFF0080FF1F9069FF1F41
:1039C0003B00010870B500252549264A26484D636D
:1039D00008CA1B051B0DED188242F9D10026802272
:1039E000224B92058B630921214B224C1E62224BF4
:1039F0001120DA67214BDA688A43DA609A68204935
:103A00000A409A60266008F057F8112008F094F8F0
:103A10008022636C93436364EE24E4006C43194A90
:103A2000200C0400642390420AD8FA223300D2000A
:103A3000904205D9144B0A21C01807F0B5FDC3B256
:103A4000124A11201372D48007F0CEFD104B1B7860
:103A5000002B04D10F4B1021187808F05DF870BDD1
:103A6000000005408805054000060540FF010000F4
:103A700000F000400038004004E100E03CF000406D
:103A8000FFDFFFFFB70B000030F8FFFF205CFF1FD8
:103A90005A5EFF1F585CFF1F002210B51100112055
:103AA00007F07AFF10BD0000F8B500230926374F54
:103AB000374C3B62E3681120B343E36008F03CF805
:103AC000112007F0F9FF112008F03EF8402322688A
:103AD00080251343236080236268DB021343636005
:103AE000A3682C4A2B43A360A36802211340A36060
:103AF0008023A2689B0113431022A360236C07203C
:103B000093432364236C0F3A1343236480235B00A5
:103B10003B62226B204B1A402263626B1A40626345
:103B2000A26B1A40A263E26B1340E363E3681B4A93
:103B30001340E36006F062FB0121072006F072FCEF
:103B4000174B11205A6C15435D6407F095FFFD215A
:103B5000144B154A89005A508023C720626B5B03BF
:103B600013436363E36880003343E3600F4B104A01
:103B700019581140802212020A431A5080229205DD
:103B80001A6008220B4B5A63F8BDC04600F0004093
:103B90003CF00040FFFFDFFFEFFFEFFFFFFF7FFF85
:103BA000003800400000FF1FC539001100E100E0AF
:103BB000FF00FFFF0000054030B503A804880B207C
:103BC000002C0ED14968074D087849780902014355
:103BD0000A20A94205D1012120001980024B1B7A3D
:103BE000137030BD192A0000205CFF1FF7B51500C7
:103BF00008AA16884A680F4F147852781202224396
:103C00000A24BA4214D10122DBB2019200962A00A2
:103C100007F05AFC041E0BD1074B1B68002B07D082
:103C200068782A7800021043424250410130984798
:103C30002000FEBD02290000A45BFF1F30B5012556
:103C400003790400BFB02B4211D00A49408806F026
:103C5000A7FF28420BD0084B01A95B8D4D800B803C
:103C6000064B00221B7A60880B7104F08FF83FB07E
:103C700030BDC0469C5BFF1FD83AFF1F205CFF1F72
:103C800010B50549054806F041FF0421044A0548DE
:103C900006F0FEFE10BDC0469C5BFF1FFFFF00004C
:103CA00014BC0011D83AFF1F10B5024804F0F0FE12
:103CB00010BDC0463D3C0011062310B58370103383
:103CC0000371443B43712A3383714433C37100232E
:103CD0000222012103720E4B027041701C88817216
:103CE0004472197A0273C1729A784273DA788273D5
:103CF0000322C2731A7902745A7942740C228274B4
:103D00009A79C274DB7903751123C370152010BD35
:103D1000205CFF1F10B5142007F04EFD124B14223B
:103D20000021186007F078FD002007F025FE012033
:103D300007F052FF022007F047FE032004F04CF981
:103D4000042006F061F9052003F08AFB062004F048
:103D500057F8072001F05AFA082006F079FE0920EA
:103D600001F034F810BDC046A85BFF1F07F0CCFE81
:103D7000012007F001FD07F0BFFC0000094B10B562
:103D80000400984205D0012904D12000064906F01C
:103D9000BDFE10BD0229FCD1013904F037FE002818
:103DA000F3D0F6E7FEFF0000CE5BFF1F70B50D7A83
:103DB000100004AA2C00168810221440154220D1AD
:103DC000002E20D10A78022A18D14A685178157835
:103DD0000E4A09022943914205D00D4A914209D069
:103DE0001C800A2404E014220A491A8007F024FCEB
:103DF000200070BD0C2208491A80F7E71C800124BE
:103E0000F6E70824F4E70B24F2E7C046F3FF0000CE
:103E1000F4FF00002C3DFF1FF0BC001110B50400A2
:103E20000749084806F072FE074804F071FD0020BB
:103E3000E40704D50721054A054806F029FE10BD10
:103E4000CE5BFF1FFFFF00007D3D001158BC00113D
:103E50001C3BFF1F00B50C4BBFB01A780B4902A8E2
:103E600000F0C2FC6B4680B2D880002809D06A46B8
:103E7000074B01A91B889380064B0022188803F08A
:103E800085FF3FB000BDC046AC5BFF1FAD5BFF1FB1
:103E9000763BFF1F803CFF1F00B50C4BBFB01A786C
:103EA0000B4902A801F0B8FE6B4680B2D88000280A
:103EB00009D06A46074B01A95B8D9380064B00220F
:103EC000188803F063FF3FB000BDC046D65BFF1FFC
:103ED000D75BFF1F1C3BFF1F803CFF1FF7B50E0089
:103EE000377A1C0008AB11003D001A8820231D40C2
:103EF0001F423CD13378022B3BD173681F785B782B
:103F00001B023B431E4FBB4208D01E4FBB4214D086
:103F10001D4DAB4221D00A252800FEBD002A2AD122
:103F2000142C2AD82200F06807F086FB174B1C706F
:103F3000012CF1D9FFF7B0FFEEE7002A1BD1202CAE
:103F40001BD82200F06807F077FB114B04211C708E
:103F5000104B187807F0E0FDDEE7E3B20124009291
:103F600001940A00310007F0AFFA0500D4E70825F4
:103F7000D2E70125D0E70B25CEE70D25CCE7C046DB
:103F8000F3FF0000F4FF000002290000D65BFF1FD2
:103F9000AC5BFF1F585CFF1F332310B50400037098
:103FA0000A220749013007F047FB064B0F201B6828
:103FB0001A0AE37222731A0C1B0E6273A37310BDEC
:103FC000205CFF1F485CFF1F30B50125037904000A
:103FD000BFB02B4213D00B49408806F0E1FD2842C8
:103FE0000DD06A46084B02A81B889380FFF7D4FFC8
:103FF0006B46D8800022608801A903F0C7FE3FB05D
:1040000030BDC046CE5BFF1F763BFF1F10B5024898
:1040100004F03EFD10BDC046C93F001170B516004A
:1040200004AA148805AA15784A6850781178000205
:104030002A4A0843801805284BD807F00DFB0313C4
:104040001E29343F0720032C0BD80422121BAA423E
:1040500000D92A0022491A803000091907F0ECFA29
:10406000002070BD0720112CFBD81222121BAA427F
:1040700000D92A001B491A80EEE707200E2CF0D841
:104080000F22121BAA4200D92A0017491A80E3E71F
:104090000720032CE5D80422121BAA4200D92A00CB
:1040A00012491A80D8E70720032CDAD80422121B01
:1040B000AA4200D92A000E491A80CDE70720032C16
:1040C000CFD80422121BAA4200D92A0009491A801B
:1040D000C2E700220A201A80C3E7C046DCD5FFFFF2
:1040E000A3BC0011F45BFF1F93BC00118EBC001138
:1040F00089BC001184BC001110B50D21024A03488F
:1041000006F0C6FC10BDC04678BC00118C3BFF1FFA
:10411000F0B50024274E85B03000B47100F0E2F80D
:10412000254D264BEA89297C9A422FD10423300061
:1041300003AA00F057F90400300000F011F9012340
:10414000B371002C34D16B4699892B68C9BA4B43A3
:1041500029891B4A1B145B1853806B46D9896B68ED
:1041600049BA89B24B4369891B0C5B181548191C65
:104170001BB2834200DD011C0B0400D50021138813
:10418000918001331380200005B0F0BD022722008A
:1041900003AB3000009700F0F7F80E230400297CF1
:1041A0000122300000976B4400F0EEF80443C3E7AF
:1041B0001C00E8E7643CFF1F085CFF1F830500004C
:1041C000205CFF1F0F27000073B5234E300000F066
:1041D00089F8224D07236A463000297C00F002F955
:1041E00004003000002C33D16B461B787F2B2FD876
:1041F00000F0B6F86B46D878F02302041B031A408F
:104200006B469B8816495BBA9BB21A432B68000920
:1042100053432A891B0C9B184B806B465A789B781A
:1042200012031B011A436B68024353436A891B0C38
:104230009B180C481A1C1BB2834200DD021C13049D
:1042400000D500220B888A8001330B80200076BDC8
:1042500000F086F80124F9E7643CFF1F085CFF1FAB
:10426000205CFF1F0F27000070B5114C237C002B32
:104270000FD0382B0ED10F4D280000F033F8CC238F
:10428000AC222800217C9B0100F0F4F8280000F00B
:1042900067F870BD084BE2899A42FAD1054D2800B3
:1042A00000F020F800222800217C00F0C5F8EDE79E
:1042B000085CFF1F643CFF1F8305000010B5084B1E
:1042C0001A7C002A09D05B69002B06D09847041E8F
:1042D00001D0FEF795FE200010BD0124F9E7C0468D
:1042E000085CFF1F70B5C17905000C00631E9C417E
:1042F0001A4BE402E41849000460C9B2007906F0E0
:10430000C7F8E979687949000131C9B206F0C0F807
:10431000E8790930C0B207F017FC0023E366613387
:104320002360AA795B3B002A0ED022689A43023BA5
:10433000134323600A23E3610733236200232363CB
:10434000A3630133E36370BD22689A4302231343DE
:104350002360462363610633A361EFE7005000400A
:1043600070B5002504000368DD66C0790930C0B26D
:1043700007F0E2FB2900207906F026F82900607991
:1043800006F022F870BD0000F8B51E0006AB1D78DF
:10439000002304681700E366616007F06DFA0123EB
:1043A0008022E3662B0027615200013B08D207F010
:1043B00063F908200A4A1168002D03D12800F8BDCE
:1043C0002261F2E7236F034203D02369013D33707A
:1043D000013613685B1A032BEED90125EEE7C046C0
:1043E0006008FF1F70B51C00002305681600EB660F
:1043F000696007F041FA01238022EB662300520036
:10440000013B08D207F038F908200A4A1168002C4D
:1044100003D1200070BD2A61F2E72B6F034203D065
:104420002B69013C3370013613685B1A032BEED9FC
:104430000124EEE76008FF1F002370B50468150033
:10444000E366616007F018FA0123E366256107F06F
:1044500013F98020064A80001168636B034205D17E
:1044600013685B1A032BF8D9012070BD0020FCE70C
:104470006008FF1F70B51D00002304681600E36686
:10448000616007F0F9F90123E36626610F33626B7F
:104490001A42FCD02B0A23611023626B1A42FCD013
:1044A000EDB2256107F0E8F88020074A8000116826
:1044B000636B034205D113685B1A032BF8D9012003
:1044C00070BD0020FCE7C0466008FF1F70B51E00ED
:1044D000002305681400EB66696007F0CDF901233D
:1044E000A619EB660F33B4420ED107F0C5F8802051
:1044F0000A4A800011686B6B03420CD113685B1A87
:10450000032BF8D9012070BD21782961696B19420C
:10451000FCD00134E7E70020F5E7C0466008FF1F44
:1045200010B5084CE368002B08D18022064B5202DC
:104530001B689B186360054B1B68236007F0FCF940
:10454000A06010BD485CFF1FC8F00040CCF00040E8
:1045500070B5184A936A916A9942FBD116498A68E4
:104560009A421FD39A1A8B60144B0126186893B293
:10457000D202D20E4343424300204C681B0A1B194F
:1045800012029B180E4C0A684B60551CA3420CD8B3
:10459000002801D04B600A600A4A136008680A4B81
:1045A000186070BD581E821ADDE7084A30009B185B
:1045B0002A00EAE700F00040485CFF1F140AFF1FD2
:1045C00040420F00C8F00040CCF00040C0BDF0FFFA
:1045D00070B51F4C23793F2B01D93F2323711D4B0D
:1045E00022791A701878C0B207F06EF818231A49A9
:1045F0001A4A0B801A4913800B805380A3791949FA
:1046000080200B800C21938001334B43164D191CE5
:104610000001834200D9011C2980D1806379002BDD
:1046200011D101336371237A012B01D80223237244
:104630006279237A0D4853430A21584306F0B4FFA8
:104640000B4D286070BDA02BEDD9A023EAE7C04632
:104650003C5CFF1F480AFF1F7E3CFF1F483EFF1FB8
:104660007C3CFF1F7A3CFF1F783CFF1F710200005B
:104670002C5CFF1FF8B514210020FEF7AFFE114C93
:10468000011E114D09D10C22104BC1CBC1C4280011
:1046900007F0C2F8FFF79CFFF8BD0C2220000C4980
:1046A000FEF770FE0C2802D0084B43CB43C40C220B
:1046B00028000849FEF766FE0C28EBD00C220021EA
:1046C000E5E7C0463C5CFF1F085CFF1FE4BC00112F
:1046D000FC0C0000F50C0000F0B51D4C8022A54438
:1046E0000400882069465201400507F0EDF9902248
:1046F00012016A441300200032C832C316C816C320
:104700008023144C144FA6689B033343A3603B6083
:1047100007F07AF88823A0685B05C01807F004FA50
:104720000025882329008022A0685B05C018401955
:104730006944520007F028F980230135FF355B01F9
:104740009D42EED1A6603E60044B9D44F0BDC04644
:10475000FCEFFFFFBC3DFF1F9808FF1F0410000087
:10476000F0B5040087B0002825D0684607F044F96A
:104770001B4C022806D106226946200007F084F966
:10478000002816D06946002301250F262F00E25C81
:10479000013310091030874038002F003240974015
:1047A0003A0002434A610439062BEFD16846FFF70D
:1047B00093FF07B0F0BD182269460A4807F084F954
:1047C0006A46A300D358013305D01822FF2168465A
:1047D00007F022F8EAE70134062CF1D1E9E7C046F8
:1047E0006509FF1F00090011F0B5002504000E0047
:1047F00085B0AA4200D186E04B1C087801934B7823
:104800008978377909021943F3783F061B040B4373
:104810001F43039720706570252800D196E033D898
:10482000112813D807F008F8690025012501250192
:104830002501AA00B800B1002501250125012501A7
:10484000250125012501250105011F01232800D18E
:10485000DEE0DB2800D02EE1042A00D8ACE01025F1
:10486000052A05D0551F2A003800711D06F0E4FE08
:1048700005223100200006F0DFFE2A003900601D0D
:1048800006F0DAFE05353EE0562859D010D8332818
:1048900000D19DE0552839D02628DAD19C4B29003B
:1048A000132218001D0006F0B7FFFEF7A9FB5CE01D
:1048B000712800D177E0722800D180E0602800D113
:1048C0008BE0DC28C5D1022A00D875E07378BFB22E
:1048D0006370B378A370032A05D0033A390092B20B
:1048E000F01CFEF789FC10223900E01CFEF74AFD9F
:1048F000C51C002807DA60705CE00C2220008549A6
:1049000006F09AFE0C25280005B0F0BD013A824D54
:104910000C2A13D8002A0AD02800019906F08CFE30
:10492000FFF756FE0C2228007C49FEF765FC2900A3
:104930000C22601C06F080FE0D25E4E70C22EBE75C
:10494000754D774B2A0043CB43C2E9E7013A704DDE
:104950000C2A11D8002A08D00199280006F06CFE14
:104960000C2228006F49FEF747FC29001322601C27
:1049700006F062FE1425C6E70C22EDE705226A491F
:10498000601C06F059FE0625BDE712226749601C2F
:1049900006F052FE1325B6E708226549601C06F0B2
:1049A0004BFE0925AFE77178F02905D8614B1888CF
:1049B00001F08EFD0225A6E7FF236370FAE75E4B48
:1049C000012A03D072789A706270F3E79B78F4E75B
:1049D0002000FFF7E1FA050095E7013A564B574DE5
:1049E000062A10D8002A10D00121280059700199F8
:1049F00006F022FE01F042F829000622601C06F0B3
:104A00001BFE07257FE70622EEE700225A70F3E738
:104A1000042A04D94A4D2F6006F08EFFA860FFF7E4
:104A200097FD0422039003A9601C06F005FE0525EE
:104A300069E7444D062ADFD906222800019907F0CC
:104A400023F80028D8D006220199280006F0F4FDAA
:104A500006223D492800FEF7CFFB0123364A917814
:104A60000B439370C8E7012AA6D07078FFF778FE51
:104A7000A0E7012800D0ECE6931E344F1A2B04D88F
:104A80007378002B09D100F015F9314B39001D78EE
:104A9000601C6A1E06F0D0FD35E7551E2A000199FC
:104AA000380006F0C9FD2B49AAB23800FEF7A4FB76
:104AB00000F036F9E9E7DA281DD1042A00D87BE7AF
:104AC000082A15D9B37972791B021343F2791204BB
:104AD0001A43337A1B0613433B603B6805223100BF
:104AE0002000039306F0A8FD0422601D03A956E7E9
:104AF000FE236370F1E7DE2800D05DE7511E012A36
:104B000001D10025FFE6019800F09EFFF9E7C046BD
:104B1000085CFF1FF0BC00113C5CFF1FFC0C000098
:104B2000E4BC0011F50C0000145CFF1FF45BFF1FD8
:104B3000C03DFF1F803CFF1F385CFF1F1D3DFF1F56
:104B4000485CFF1F6509FF1FADAC0000395EFF1F09
:104B5000375EFF1FAEDE000070477047020010B5E1
:104B6000094B0A32094C92B2DA815A829881188232
:104B7000207802F013FB0422054B012120781A70E3
:104B800006F0CAFF10BDC0464A3DFF1F825EFF1FF0
:104B9000815EFF1F013870B5042809D806F05CFD5E
:104BA000030928081200234B0221187806F0B4FFED
:104BB00070BD204B0821187806F0D6FF00221E4B4E
:104BC0001A72F5E7802200241B4B1A4D52001A81FD
:104BD00008211A682878DC7206F066FF2100287820
:104BE00006F0BAFF012000F067FE00F047FFDFE7A4
:104BF000104B0821187806F0B7FF1048FFF75CF853
:104C00000F4B104A9B79002093800F4A138080221B
:104C1000094B5200D8721A8100F04EFE00F02EFFB0
:104C20000A4B9B78002BC3D0094A136006F0FCFEA8
:104C3000BEE7C046585CFF1F2C5CFF1F893CFF1F6E
:104C40003C5CFF1F483EFF1F7A3CFF1F385CFF1F84
:104C500034F0004010B501290BD1082809D1054BCB
:104C60001B78002B05D02622034B04485A72FFF70D
:104C700075FF10BD5A5EFF1F2C5CFF1FC4090000AA
:104C80000300F0B50A4D8E18B14202D152008018CF
:104C9000F0BD0C782F6824093C5D0F271C700C7840
:104CA00001313C402F683C5D5C700233ECE7C0464C
:104CB000743CFF1F0D22114B10B51A700C23104CC1
:104CC00010492370093A033B0F48637006F0B4FCA7
:104CD0002D2301220D490E48A371FFF7D1FF0122B8
:104CE0000C49FFF7CDFF01220B49FFF7C9FF002256
:104CF0000A491000FEF780FA10BDC046565EFF1F3D
:104D0000375EFF1FA3BC0011395EFF1F6709FF1F3D
:104D10003E5EFF1F6609FF1F6509FF1FAEDE000034
:104D200070B5124C132220001149FEF72BFB114DD8
:104D3000002817DDAB78002B14D0431C2B700923FF
:104D40006B70002300190370287829000130C0B26D
:104D500006F0F2FC297822000139C9B2002005F0E2
:104D6000B5FD70BDFFF7A6FFEEE7C046395EFF1F39
:104D7000AEDE0000375EFF1F10B5114B1A781870B9
:104D8000002A0ED000280BD10E4B1A78062A07D81D
:104D90005423D340DB0703D50B4B187802F0FEF900
:104DA00010BD0028FCD0074B1B78012B02D0033B21
:104DB000022BF5D8044B0121187806F0ADFEEFE781
:104DC0005A5EFF1F815EFF1F825EFF1F70B5514E4E
:104DD000514A52493070082005F01AFC0121022086
:104DE00005F020FB022005F001FC0121002005F068
:104DF00019FB002005F0FAFB00F0AAFEFEF700F90F
:104E000006F0C2FE032246494648FFF739FF2D242B
:104E1000030004221C7044490130FFF731FF3023A6
:104E20000470424D424C437083702E3B062220009A
:104E30004049EB87FEF7A6FA062813D0200006F0BB
:104E4000DBFD022809D00321200006F0D5FB8D23CD
:104E5000E3706E3B237119336371062220003549DC
:104E6000FEF7CAF9344B1B68FC335C64FFF758FF4C
:104E70000020FFF781FF314C314A0121314B12787C
:104E8000207802F04DF9304A304B1278002120781A
:104E900002F046F901222E4B1A702E4BDB78552B6F
:104EA00031D12D4B3B325A722C4B2D4AAB81EA81CA
:104EB0002B826A822021307806F02EFC01204042AD
:104EC00005F050FD0120404205F0ECFDFFF714F91C
:104ED000FEF7D6FE00F0A4FC01204042FEF79EFF44
:104EE000012006F0D1FBF02001F0D6FA0121307844
:104EF00006F012FE307802F0ADFA1A4806F0DCFC3B
:104F0000FEF7D2FD70BD6422174B5B7953431A0044
:104F10000A32CBE7585CFF1F594B0011554C00116A
:104F2000C03DFF1FF45BFF1F145CFF1F4A3DFF1FC6
:104F30006509FF1FADAC0000AC5EFF1F825EFF1F66
:104F4000A83CFF1F893CFF1F565EFF1F375EFF1FF7
:104F5000285EFF1F385CFF1F2C5CFF1FC409000088
:104F6000CE0900005A5CFF1F3C5CFF1FF8B50A0029
:104F700020230D001A40194257D0574B1B78002BA5
:104F800050D0FFF7E5FA554B554C564E996862687C
:104F9000737A8A1ADB039A4202D36160FEF784FDBA
:104FA000327A217A531EDBB2994205D1FFF75CF9C0
:104FB000002000F099FD0FE09142F9D30023237205
:104FC000FFF77CF9012000F08FFD474F3800FEF716
:104FD00073FE390006F0F8FD637A002B1FD0013B09
:104FE000DBB26372002B1AD1404BDB78552B01D119
:104FF00006F01AFDE37A002B0CD000233C4A3A4F0E
:10500000E3721388380001331380FEF755FE390030
:1050100006F0DAFD642370795843FFF79FFD237A89
:105020000133237220206840F8BD0BB2002B0ADA4E
:10503000304B187806F018FD002801D006F09CFDD2
:1050400080200002EFE70224214206D0244B0120F9
:105050001A72FFF791FE2000E5E70B071ED5FFF758
:1050600077FA1E4B1E491F4C98684A68637A821A69
:10507000DB039A4202D34860FEF716FDFFF71EF9E4
:10508000FFF7F2F8012000F02FFD00F0E3FB2368AA
:10509000DB0701D5FEF7BAFF0820C4E71024214240
:1050A00006D00D4B1B78002BD5D1FEF7FDFDD2E7C6
:1050B0000124214207D0104800F06CF806F07CFA79
:1050C00000F0F8FCC7E70424080020402142ABD0E0
:1050D000FEF7C0FEBFE7C0465A5EFF1F485CFF1FD9
:1050E0002C5CFF1F3C5CFF1F893CFF1F385CFF1FCF
:1050F000205CFF1F585CFF1F6C3CFF1FF0B51B4B73
:105100001B4F1B883A8804001A4E1B4D85B09A42EB
:105110000DD832889A420AD3184B1A882B889A42A3
:1051200005D1174A174B12881B889A421BD00520BD
:1051300001F008FA3B8802AA13803388019053805B
:105140002B88114D93800F4B02A91B88D3800F4BE6
:105150002A78188802F024FF0D4B08212878019A3C
:105160001C7006F019FA05B0F0BDC046265EFF1FA0
:105170007E3CFF1F7C3CFF1F7A3CFF1F245EFF1F0D
:10518000225EFF1F783CFF1F825EFF1F803CFF1FD7
:10519000205EFF1F13B50C4B1C78002C11D100288A
:1051A00001D00A4B18600A4A0A4B11780A4A107853
:1051B0000A4A01920A4A0092002205F07FFA200072
:1051C00016BD1124FBE7C046815EFF1F1C5EFF1F5A
:1051D000805EFF1F705EFF1F825EFF1F5C5EFF1F11
:1051E000605EFF1F10B5064B12201B78052B06D101
:1051F000044B13221988044B187801F07FFB10BD73
:10520000815EFF1F803CFF1F825EFF1F10B50024E0
:105210000122114B52421870104B1C70104B1A8017
:1052200002F018F904220F4B21001A700E480C32BC
:1052300006F09AFA102221000C4806F095FA07228F
:105240000B4B1C600B4B1C700B4B1C700B4B1A70E8
:105250000B4B1C7010BDC046825EFF1F815EFF1F9E
:10526000803CFF1F805EFF1F705EFF1F605EFF1FA0
:105270005C5EFF1F365EFF1F355EFF1F823CFF1F17
:10528000345EFF1FF8B5174C0600257806A81424D5
:105290000078052D23D1B41F134FA5B21824BD42A9
:1052A0001DD88D1FADB2BD4219D8FA256D00AA4296
:1052B00015D21D000D4F0A3DADB2BD420FD80C4CAA
:1052C00026800C4C21800C4900240A800B4A138054
:1052D000FFF714FF0A4B0421187806F045FC200064
:1052E000F8BDC046815EFF1F790C0000750C000000
:1052F0007E3CFF1F7C3CFF1F7A3CFF1F783CFF1F5A
:10530000825EFF1FF0B50BB20D0089B0002B00DBF1
:1053100070E1A44E307806F0A7FB041E50D003784D
:10532000A22B00D122E1D02B1AD0912B45D143786A
:105330000E2B42D19C4B82889A423ED19B4A836875
:105340001278052A39D1032018567F2835D0984B7A
:105350001B68002B31D05B68002B2ED098472CE0C7
:105360008078072829D806F077F90428183F3F7479
:10537000A8D86378002B0CD101218C4B19708D4B70
:105380001A78002A5BD08C4B307801F0C9FE0028D7
:1053900055D00722854B1A7051E061780029F8D169
:1053A000E378002B11D0854A854B1278307801F0D4
:1053B000B7FE60706378002BEBD1200006F0DCFBB9
:1053C00080200002684009B0F0BD784B1B78022BAA
:1053D000F3D00121307806F007FB0028EAD1012143
:1053E000307806F099FBE5E76378002BD1D16F4F59
:1053F000032807D13B78052B02D101333B701EE017
:105400000223FBE76F4B1A886F4B0293002A0BD0E5
:105410001B78002B03D00121307806F0BDF83B78D3
:10542000062B04D1013BE9E7029B1A70F7E7042B36
:1054300041D10121029B3078197006F06DFB5C4B65
:105440001B68002BB9D01B68002BB6D0574A1078C8
:1054500084E76378554F002B27D10622211D5B4836
:1054600006F0EAF862895A4B5A491A80A2895A4BC7
:105470001A80E3890B800521397058490A80584AFF
:105480001380228A574B1A80574B1B78012B09D166
:105490001F2001F057F8FA2292004243042130788D
:1054A00006F07AF80022484B75E7312B00D070E700
:1054B0000022454B1A700323A0E70622002143482F
:1054C00006F052F90023454A04211380444A3078FB
:1054D0001380444A138006F047FB0821307806F019
:1054E00043FBA379083B5A425341304A03331370BC
:1054F000304B1B78002B06D0334B30781A78002ABB
:1055000006D001F04BFE0122314B52421A8096E741
:105510000121197006F000FBF5E70821307806F04C
:1055200023FB6378002B00D047E72C4B2D4F0293D1
:10553000E388029A04211380294B3078039323894E
:10554000039A138063893B8006F04EFA002800D04E
:1055500033E7264B1B68002B00D12EE703990298F6
:105560003A88098800881B68984726E74379132BF7
:1055700000D022E70389012B0AD11D4B1B78022B97
:1055800006D10821307806F0EFFAFFF72BFE14E77A
:10559000052000F0D7FF08210200307805F0FCFF5D
:1055A0000BE7C046825EFF1F05140000815EFF1FEF
:1055B0001C5EFF1FA83CFF1F893CFF1F565EFF1F9C
:1055C000375EFF1F585EFF1F5A5EFF1F295EFF1FD9
:1055D000803CFF1F305EFF1F325EFF1F265EFF1FF5
:1055E000245EFF1F225EFF1F285EFF1F185EFF1F45
:1055F000205EFF1F8020C001014200D0E2E6CB0701
:1056000031D5324B1B78002B1DD0314E05AC337891
:10561000052B1AD1023B23702E4B21001B782372DD
:105620002D4B1B7863722D4B187801F01DFD00285F
:1056300009D007202A4B30701B68002B03D01B6851
:10564000002B00D098470120BCE60E20254B0622F7
:105650001B7825492370254B1B78637002ABC0185B
:1056600005F0EAFFD8E7022308001840194209D0E4
:10567000174B1B78052B03D11D4B188805F0ACFF89
:1056800002209FE60424214203D0FFF737FD2000CB
:1056900098E6082308001840194200D193E6154BFC
:1056A0001C78012C03D0022C0DD008208AE6124B66
:1056B000124A134913481B881288098800880094ED
:1056C000FFF7E0FDF1E7FFF78DFDEEE75A5EFF1F04
:1056D000815EFF1F823CFF1F345EFF1F825EFF1F43
:1056E0001C5EFF1F365EFF1F833CFF1F355EFF1FE2
:1056F000803CFF1F205EFF1F783CFF1F7A3CFF1F8E
:105700007C3CFF1F7E3CFF1F10B502A804880B20C5
:10571000002C10D1496808784978090201430C48E7
:10572000814209D1022119800A4B59881170DB7816
:1057300000205BB2537010BD074C0A20A142FAD181
:1057400002211980034B998811705B79F0E7C046FC
:105750006E2A0000205CFF1F6F2A0000F7B51500BD
:1057600008AA16884A680F4F14785278120222430A
:105770000A24BA4214D10122DBB2019200962A0017
:1057800005F0A2FE041E0BD1074B1B68002B07D0AF
:1057900068782A780002104342425041013098470D
:1057A0002000FEBD02290000945EFF1F30B50125D8
:1057B00003790400BFB02B4225D01449408805F07E
:1057C000EFF928420CD0124B01A95B8D00220B800F
:1057D00002234B800F4B5B888B80608802F0D6FAE7
:1057E0000D49608805F0DCF9C0070CD50B4B01A909
:1057F0001B8800220B8002234B80064B9B888B80EA
:10580000608802F0C3FA3FB030BDC0468C5EFF1F17
:10581000AC3CFF1F205CFF1F845EFF1F063DFF1F87
:1058200010B5074C0749200005F070F92000064923
:1058300005F06CF90721054A054805F029F910BD66
:10584000FFFF00008C5EFF1F845EFF1F10BD001174
:10585000AC3CFF1F10B5024803F01AF910BDC0465A
:10586000AD57001170B55F25082607498400CA7836
:105870008B7840012A40B3433440A843234302437A
:105880008B70CA7070BDC0461D3DFF1F010043B242
:1058900004205A0002409B000C3003401A43152399
:1058A00010B5044CE0789843143B0B401843024376
:1058B000E27010BD1D3DFF1F10B5054B082419797E
:1058C0000A00A243002801D022000A431A7110BD29
:1058D0001D3DFF1F10B5054B4024D9780A00A24397
:1058E000002801D022000A43DA7010BD1D3DFF1FC1
:1058F0000821F8B5324D334BAE7804000E40AE703F
:10590000984204DD67232B70473B6B70F8BD2E4B2C
:10591000984203DAE0232B703A3BF6E700232B7022
:105920006B7083B21A0029485F3292B2284F8242CC
:105930002CD9002C03DA5B421CB204232B700534F3
:1059400020B20A2105F030FE04B2FA239B009C42EB
:1059500032DB08232A7813432B706421200005F0E2
:1059600023FE0A2100B205F06FFE09B22A787B5CA3
:1059700013432B700A21200005F016FE0A2100B205
:1059800005F062FE09B27B5C6A780AE06970002C5F
:10599000DBDA5B421CB204232B70F3226B78092CF8
:1059A000E8DC13436B700A21200005F04DFE09B2BC
:1059B0007B5C1E43AE70A9E7632CCEDCEDE7C046EE
:1059C0001D3DFF1F1B4E00001DFCFFFF2A080000AD
:1059D0003ABD00110823F7B5194FCD003E790400F8
:1059E0001E403E71EDB2632806DD5F3333433B71E9
:1059F00020231D437D71F7BD0300093305DA202301
:105A00005B4233433B71A623F3E70E4B019300281F
:105A10000BDA0423444224B23B710A21200005F032
:105A200013FE019B09B25B5CE3E70928F5DD0A215F
:105A300005F0BAFD019B00B21B5C1E433E71ECE712
:105A40001D3DFF1F3ABD0011F8B50A4F05003B7818
:105A50000E00002B0CD0084C2000FEF743FC330056
:105A60002A0020003978FEF731FD2000FEF778FC8F
:105A7000F8BDC0469F5EFF1F243DFF1F70B50A4E54
:105A80000A4D06223100280005F0FEFF002809D04B
:105A9000074C31000622280005F0CEFD072120002A
:105AA000FFF7D2FF70BDC0461D3DFF1F995EFF1F6F
:105AB000985EFF1FE622402110B50A4B1A70403A4B
:105AC0005A703E329A70DA780A40DA7008221979F0
:105AD0001140053A0A431A7147225A71FFF7CEFF67
:105AE00010BDC0461D3DFF1F10B500282AD0164C22
:105AF0000A210223E05E05F057FD00B2FFF7F8FE31
:105B00000423E05E642105F04FFD012100B2FFF7A0
:105B100061FF237A0024132220009A426041C0B220
:105B2000FFF7D8FE0320FFF79DFE2000FFF7AEFE33
:105B3000064B1878053843425841C0B2FFF7BCFE07
:105B4000FFF79CFF10BDC046205CFF1F815EFF1F5A
:105B500070B500250A4C2000A571FEF7C3FB102389
:105B60003E212000074AFEF7B1FCA84200D13E3595
:105B7000054B20001D70FEF7F3FB0123A37170BDE0
:105B8000243DFF1F2ABD00119F5EFF1F0200F0B5DC
:105B900001270A480A4E51188B1A002B00DCF0BD71
:105BA000082415784308684038404000805B013C79
:105BB00058406D08002CF5D10132EDE7FFFF0000E1
:105BC0004ABD0011F0B500250F269D4200DBF0BD57
:105BD0004C5D070944403440A400A058013578408A
:105BE000F3E70000F0B589B06A460D000B000F27FF
:105BF000110010351C780133260024093E40167030
:105C000054700232AB42F5D12023024AFFF7DAFF8B
:105C100009B0F0BD50BD0011F0B54E780B7889B0D9
:105C200036020C00170001901E43012A61D9954BE2
:105C30009E4200D877E001339E421CD1062A17D13C
:105C4000CA788B7812021A430B791B0413434A79E2
:105C500012061A438C4B5A6100221A705A808B4AE2
:105C60005A608B4A9A608B4ADA60002009B0F0BD16
:105C700088225205EEE7884B9E423CD182498B78C0
:105C8000002B00D0F6E00C2A31D10F22A3789343E9
:105C9000E278120213432279120413436279120646
:105CA00013434B60E279A07912020243207A000488
:105CB0001043627A12060243CA60E27AA07A1202A4
:105CC000024376484A81834208D804236E4914224D
:105CD00001980B7005F0B0FC1420C7E71201D21830
:105CE00089235B059A42F0D801238B70BDE7022A15
:105CF000FAD00523EAE76A4A01239642E6D1FFF784
:105D000071FA052F0CD9E378A2781B02134322798C
:105D100012041A4363791B061343624A0393136008
:105D200005F082FEA1E7584D2B78002B9DD1AB7872
:105D3000002B00D1A0E02B8901339BB20093B3422A
:105D400000D091E0132AD4D9CF7C8B7C3F02122162
:105D500020001F43FFF71AFF874200D08EE0002E7D
:105D60003DD1E378A2781B0213432279E96812043B
:105D70001A4363791B06134303930A228B4212D101
:105D8000FF23A370E370237163716B89002B09D12A
:105D9000E37B227C1B0212041343A27B13431B09E7
:105DA00001336B8100226B89002B8ED0002A67D1D2
:105DB000686837013818000B6B690003039098423C
:105DC00005D9686105F0B0FEEB780133EB706868C7
:105DD0001022A11C381805F0D7FD2E8145E76F89E8
:105DE000009A7B1E9BB293423AD1E278A3781202CA
:105DF0001A43237905A81B04134362796C681206C1
:105E00001A43EB6800920392211D0C22049305F0C3
:105E100013FC0120260004A940421036FFF7E2FEE1
:105E2000013F012F17D1009A0B232861824200D035
:105E30004CE704221C49200005F0A6FD042203A91A
:105E4000686805F041FEE968039AFF23914200D19A
:105E50003CE7F73B3AE73100FFF7C4FE1036DFE7D7
:105E60000923B742A4D831E7009BB34200D9FCE62E
:105E700007232BE7022329E7032327E7062325E748
:105E80000A2323E7FFFE00002C3DFF1F0000011145
:105E9000FFFF00005048593601FF0000FFFF0011CE
:105EA00002FF000034F00040383DFF1F10B5034CE6
:105EB0000B000122210000F06BFA10BD6D60001193
:105EC0000B8870B506000D000224162B11D92B008B
:105ED0000322094900F05CFA041E0AD1074B2A8804
:105EE0001B88191C934200D9111C300089B200F0A4
:105EF000EFFA200070BDC04699600011C65EFF1F1A
:105F000010B54A780400013A0B000220012A07D894
:105F10000A78002A04D005222000024900F038FA4D
:105F200010BDC046C76000110A7810B50B00040010
:105F30000220002A04D007222000024900F028FA9B
:105F400010BDC046736100110A7810B50B00040043
:105F50000220002A04D009222000024900F018FA89
:105F600010BDC046D961001110B5034C0B000B22C7
:105F7000210000F00DFA10BD0962001110B5034CAC
:105F80000B000D22210000F003FA10BD7B6200110E
:105F900010B5034C0B000F22210000F0F9F910BDE1
:105FA000D56200110A7810B50B0004000220002A07
:105FB00004D011222000024900F0EAF910BDC046C9
:105FC000E5620011002310B51322190000F0E0F97A
:105FD00010BD000010B5034C0B001722210000F08B
:105FE000D7F910BD37630011002310B5192219002D
:105FF00000F0CEF910BD000010B5034C0B001B22C1
:10600000210000F0C5F910BD71630011F7B5848956
:106010000D0006000121002C22D000238268D356F7
:106020001778002B1EDA0C2C1AD90C3CA4B21319C9
:1060300040880093230002F086FE431E9841013001
:106040007B06DB0F6B703F23013C1F40A4B228701E
:10605000AF70AC80002C07D0B3680133AB60002177
:106060000800FEBD0020EBE7AC60F8E70B7803709A
:106070004B8843704B881B0A83700B79C3700420D4
:1060800070470420022B06D10020537811781B02A0
:10609000009A0B43138070470B8803700B881B0A10
:1060A0004370022070470420009983420AD153783C
:1060B00010781B0203430B80D37890781B020343B4
:1060C00000204B807047F8B50D004B78012400216B
:1060D000461C03702B788B4201D82000F8BD6B78EA
:1060E000B01C4F1C012B10D1890069184B8802226B
:1060F00033704B88B9001B0A7370691805F0FCFCFB
:1061000004360434A4B2F9B2E4E7122359436B18FD
:106110005A88043132705B8810221B0A7370691828
:1061200005F0EAFC12361234ECE770B5049D140059
:106130001E00052B01D8042070BD637812781B0265
:1061400013432B80E378A2781B02134302226B8057
:106150002A71211D681D063E05F0CEFCB2B22A81CF
:10616000E92AE8D82800A11D0A3005F0C5FC002066
:10617000E2E7002310B50A789A4201D8900010BDDA
:106180009A008A185488013304705488DBB2240AB8
:106190004470948884709288120AC2700430EAE7CE
:1061A00010B51100029C062B04D004201022142BE1
:1061B00001D010BD022222714B7808781B020343E4
:1061C0002380CB7888781B02034363800431601DF1
:1061D00005F092FC0020ECE710B50C788B780431C8
:1061E0005C43E4B203702200013005F085FC601CC2
:1061F00010BD0420022B06D10020537811781B0219
:10620000009A0B431380704710B50C000A880231C6
:1062100005F072FC208810BD70B504000D000498D4
:106220001100012B01D8042070BD1678527812029B
:10623000324302800200F13255701470E125002CC7
:1062400000D10C35023B9AB24280AA42EBD802310F
:10625000043005F051FC0020E6E704200099834259
:106260000AD1537810781B0203430B80D3789078BF
:106270001B02034300204B80704710B50C000A88B6
:10628000023105F039FC208810BD000070B50121F5
:106290001E000420049C0E400B4218D1CB40DDB2FE
:1062A0008D4214D90A49DBB2098899420FD32300E1
:1062B000EE331D703300580011184978165C09023E
:1062C000314301332152D9B28D42F4D8002070BD40
:1062D000443DFF1F10B50C000A88023105F00CFC8C
:1062E000208810BD10B50C788B7804315C43E4B283
:1062F00003702200013005F0FFFB601C10BD10B5DB
:1063000011000298032B01D8042010BD1478527894
:10631000043B120222430280CA788C781202224384
:1063200042809AB28280EB2AEED80431063005F022
:10633000E3FB0020E9E710B50C000B8803700B8825
:106340001B0A43704B8883704B881B0AC3708A8872
:106350000430063105F0D0FBA088043080B210BDB7
:106360000420012B03D100201378009A137070478A
:1063700010B50C000B8803700B881B0A43704A8809
:106380000230043105F0B8FB6088023080B210BDE5
:10639000F0B589B003931E4B029242000700D05A19
:1063A000019102F020F81325061E2DD0029B012436
:1063B0000370019B002B04D0001903999847001922
:1063C00084B26B461B7A5BB2002B0FDA10213800C7
:1063D00002F01CFB1925002813D130003219E1B25C
:1063E00002F066FC051E0CD10C34A4B2042304AAEE
:1063F000380005A993800696948101F0AFFD051E33
:1064000002D0300005F090FA280009B0F0BDC04677
:10641000C45EFF1F70B505000C0000280CD00020E2
:10642000814209D010222000044905F065FB0120BB
:106430002B7823736B78637370BDC04690BD0011D9
:10644000F0B506000D0017001C0085B002291BD016
:106450000020102907D1022B07D0102B03D115E003
:106460000020102C08D005B0F0BD69463800FFF7B9
:10647000D1FF2A0069460BE069463000FFF7CAFFEA
:1064800022006946380004E0022BE9D12A003900D5
:10649000300005F021F9E6E7031CF02800D9F023CD
:1064A000032008499AB2013A0B80D31703400649EA
:1064B0009B189B100B80D30F04499B185B100B801B
:1064C0007047C046483DFF1F463DFF1F443DFF1F2C
:1064D000034B1B888B4202D3024B4000C1527047D2
:1064E000483DFF1FC45EFF1F014B4000185A704714
:1064F000C45EFF1F1722014B1A807047C45EFF1F46
:1065000070B505000E2005F0FFF8041E13D0D0234F
:10651000037000230622837007494570033005F09D
:10652000EBFA064B2100DA8A62811B7E2373044B4F
:10653000187805F0D9F870BDE05EFF1FD05EFF1F30
:10654000983DFF1F262803D8024B4000C05A7047D1
:106550000148FCE74A3DFF1FFFFF000070B5060041
:106560000C00094D1C220021280005F0FDF8074B06
:106570001E70074B1C7005F08FF90123002801D015
:10658000002312202B7070BDD05EFF1F983DFF1FAF
:10659000F15EFF1F70B505000D4C0800E260A160C0
:1065A00010220021656005F027F9012803D1102190
:1065B000A06802F058FD10220021280005F01CF907
:1065C000012803D11021606802F04DFD70BDC04666
:1065D000D05EFF1F70B5041E05D1002903D006222E
:1065E0000D4805F089FA0D4B1D78012D11D1002CB5
:1065F00005D102221A7004F0E7FF280070BD0022C6
:106600001A70074B1B78FF2BF7D02000FFF778FF9D
:10661000F3E70025F1E7C046E05EFF1FD05EFF1FF5
:10662000983DFF1F030010B5002801D1002010BDC8
:1066300000780B4A002803D15988D1821B79137640
:106640001378022BF2D10023984200D10333137048
:10665000044B1B78FF2B01D0FFF752FF0120E6E728
:10666000D05EFF1F983DFF1F002911D000280CD0DD
:106670004B79012803D140225242134303E03F22C9
:106680001340032802D001204B7170474022F4E7E9
:106690000800FAE770B5094D0100287800280BD0F2
:1066A000074C0622200005F027FA21002878FFF782
:1066B000DBFF200004F0B8FF70BDC046F05EFF1F96
:1066C000CA5EFF1F00290AD0012808D13F224B795A
:1066D0009343C02B03D0403B5A425341981C704710
:1066E00070B5174D06002B78FF2B15D00A2005F04A
:1066F0000BF8041E10D0D0230370C83B8370114BDD
:1067000011491B784670C3700622043005F0F4F975
:106710002100287804F0E8FF0C4B1B78012B0DD1E9
:106720000B4B1B68002B03D09B68002B00D09847B5
:10673000084B04211878084A05F0B6F970BDC04628
:10674000983DFF1FF05EFF1FCA5EFF1FEC5EFF1F3C
:10675000185FFF1F1C5FFF1F60EA0000014B986875
:106760007047C046D05EFF1F014BDB68186870475A
:10677000D05EFF1F074B10B5DA6813680133136052
:10678000054B1878FF2803D08021C90105F0C4F912
:1067900010BDC046D05EFF1F983DFF1FF7B50E002D
:1067A00002F0C8F8051E1CD00E4B06621F78002FA1
:1067B00000D10778AB791020019304F0A5FF041EE7
:1067C0000FD0D0230380C73B8370019BE91DC370AA
:1067D0000622043005F090F921003800E66004F04C
:1067E00083FFF7BD963DFF1F014B18787047C046E9
:1067F000F05EFF1F054B002805D1054B1A78054BAD
:10680000002A00D1014B18007047C046E05EFF1F10
:10681000F05EFF1FCA5EFF1F014B58687047C046FD
:10682000D05EFF1F024B1868431E9841C0B27047EC
:10683000F45EFF1F421E03000120152A03D9FF3B0F
:106840005A425341D8B27047F0B51C0000230E00E5
:1068500085B0039002920B70029A934201D30020FC
:1068600019E0E55C5A1CD2B2002DF8D002985119FB
:106870008142F4DC0233DFB2A35C18000193FFF71E
:10688000D9FF002807D0013D019A0399EBB233707C
:106890008A4202D1E01905B0F0BDDB19DBB2DBE7BB
:1068A00010B50C0002F09EF803001220002B03D05C
:1068B0002100588804F0B8FF10BD000070B50E4DDF
:1068C00084006359002B15D0186A002801D004F009
:1068D000EBFF2B59586A002801D004F0E5FF2B5933
:1068E000986A002801D004F0DFFF285904F0DCFF8B
:1068F00000232B5170BDC046005FFF1F1C4B70B5BD
:1069000004000E00150099420AD11A4B1B68002B97
:1069100001D1122070BD1B68002BFAD09847F9E70F
:10692000154B994215D1134B1B68002B0AD01B68DD
:10693000002B07D09847002804D1104B1C70104B37
:106940001D70E7E729002000FFF7AAFF0028E1D12A
:10695000F3E7080001F0EEFF0028DAD00378032007
:10696000A342D7D12900300004F05EFFD2E7C04631
:10697000FEFF0000FC5EFF1FFFFF0000F95EFF1F2F
:10698000F85EFF1FF7B50400808801F0D3FF0025F3
:10699000A84203D00578A08802F008F81C4E33788E
:1069A000002B1FD0AB421DD11A4B28001978FFF7DE
:1069B00077FF002818D000233370A3790820A77828
:1069C000A688019304F0A0FE011E0DD0D023037011
:1069D000CA3B8370019B477086808371280004F056
:1069E00083FE01E0002DE8D1A0880B4B8200D35834
:1069F000002B01D0FFF762FF1721A088FFF768FD89
:106A0000A08801F027FDA08801F0FEFDF7BDC0467B
:106A1000F95EFF1FF85EFF1F005FFF1FF0B587B034
:106A20001D000CAB1B88070001930DAB1B881420C5
:106A300002930EAB1B88160003930FAB1B880091CB
:106A4000049310AB1B88059304F05EFE041E1AD05D
:106A5000D0230370CB3B47708370C6700622290099
:106A60000430002D11D005F047F8019B210063810F
:106A7000029B0098A381039BE381049B2382059BD7
:106A8000A37404F031FE07B0F0BD04F06DFEECE736
:106A9000F7B5009308AB1B8807000C200D0016000B
:106AA000019304F031FE041E13D0280001F042FFD0
:106AB00000280FD00078D0232370C93BA370009B1F
:106AC00021002381019B6770A580E680638104F02B
:106AD0000BFEF7BD014B1878EDE7C046983DFF1F50
:106AE00013B5040064890389C2888188C078009442
:106AF000FFF7CEFF13BD000010B5044C206800283E
:106B000003D004F0D1FE0023236010BD045FFF1FFB
:106B1000A122F0B5818892004A43384B384F1B6858
:106B200004009B189D2292009B18827989B01A60FC
:106B30003B68002B5FD01D78324B1B68002B04D0C4
:106B40005B68002B01D000209847260008363100F2
:106B5000E079FFF7B7FD237DE0710200E078049350
:106B6000638A29000393238A0293E3890193A3880C
:106B700000933300FFF752FFE378002B0BD1E2893B
:106B8000A379A18802920196E2792800009201225D
:106B900001F0DAFEE0703B68002B20D0FFF7ACFF7D
:106BA000194D287800281AD0184B1978FFF778FE6D
:106BB000002814D02B78E67808200793A78804F0E3
:106BC000A3FD011E09D0D0230370CA3B4670837019
:106BD00087808671079804F087FD00232B701721AA
:106BE000A088FFF775FCA08801F034FCA08801F0B4
:106BF0000BFD09B0F0BD064B9DE7C0463409FF1FF1
:106C0000045FFF1F185FFF1FF95EFF1FF85EFF1F85
:106C1000983DFF1FF8B5070008000E0001F08AFE3E
:106C2000041E18D02620FFF78DFC051E00D1257804
:106C3000062004F069FD041E0DD00021062204F098
:106C400093FDD0232370C23B21006770A370A68000
:106C5000E8B204F049FDF8BDF0B585B001930AAB88
:106C60001B78070002930BAB1B7808000D00009205
:106C7000039301F05FFE061E22D0102004F044FDB5
:106C8000041E1DD01022002104F06EFD2620FFF707
:106C900059FC002800D13078D0232370C13BA37069
:106CA000009B21002372019B67706372029BA58089
:106CB000A372039BC0B2E3720C9BE36004F014FD6B
:106CC00005B0F0BDF7B50D00019001F033FE071ED1
:106CD00020D00E2004F018FD041E1BD02620FFF744
:106CE00031FC061E00D13E78D0232380C53B06220E
:106CF000A370F91DE01C04F0FFFE019B2A006381D4
:106D00000123DD401A401D40210022736573F0B25B
:106D100004F0EAFCF7BD0000F0B585B00290100069
:106D20000D0017000A9E039301F004FE041E31D0EB
:106D3000029B002B2ED1039B02795B0724D51223E3
:106D400013430422002E08D10B99002905D10C9978
:106D5000002902D10D9900291AD01A430D9B2271E6
:106D6000002B00D0C9E0002E00D1CFE0002D00D0D4
:106D7000CCE0606A002801D004F096FD1C213000B0
:106D800004F08AFE606205E002239A430E33D7E7DF
:106D900093432371654BBA00D458002C00D1AAE06C
:106DA000002E10D0236A002B03D11C2004F004FD18
:106DB00020625E4BBA00D358186A002803D01C2208
:106DC000310004F099FE0C9B002B12D0574CBB00F5
:106DD0001D596B6A002B03D1162004F0EDFC68628C
:106DE000BB00E358586A002803D016220C9904F01F
:106DF00083FE0D9B002B11D04C4DBC006659B36A2D
:106E0000002B03D1142004F0D7FCB0622B59986AF0
:106E1000002803D014220D9904F06EFE380001F012
:106E200089FD051E67D0414BBA00D358002B62D0B4
:106E30001A6A3420002A00D11C389A6A002A01D02C
:106E4000143080B20B9A002A01D01C3080B25B6AE9
:106E5000002B01D0163080B204F056FC041E4AD03C
:106E60001822002104F080FC2620FFF76BFB019024
:106E7000002801D12B780193D0232370029B20009E
:106E800063700A23294EA370039BBD00A371AB5905
:106E9000A780196A1830002905D01C22A06004F0D0
:106EA0002BFE200034307359996A002907D0030063
:106EB00014221433E060029304F01EFE02980B9B30
:106EC000002B08D003001C221C330B992061029375
:106ED00004F012FE02987359596A002903D0162251
:106EE000606104F009FE6B462100187904F0FCFB98
:106EF0003800FFF7E3FC05B0F0BD10220D9B0D99A3
:106F00001B69A018236204F0F7FD2CE70B9B002BF4
:106F100000D13FE7012D00D03CE7606A002801D096
:106F200004F0C2FC1C210B982AE7C046005FFF1F3B
:106F300010B5044C2068002803D004F0B5FC0023F1
:106F4000236010BDF45EFF1F0B4B07B51A68002AC3
:106F500001D100200EBD6946531C01201278073173
:106F6000FFF772FC0028F4D00278012310001840CB
:106F70001A42EED0EEE7C046105FFF1FF0B51F4F7C
:106F800001203B6887B0002B25D09B78059300F04B
:106F9000B3FB002821D00A20FFF7D4FA04000B200D
:106FA000FFF7D0FA164B05001E78731E9E413B6812
:106FB000F6B2191DD878FFF757FB3B682900DA7A3B
:106FC000043303929A7901930292009033002000D7
:106FD000059A04F001FD07B0F0BDFFF7B5FF0028EA
:106FE00005D00620FFF7AEFA04000720D8E70820F6
:106FF000FFF7A8FA04000920D2E7C046F45EFF1F9D
:10700000F05EFF1F70B50A4E040033780D00FF2BB1
:107010000DD0042004F078FB011E08D0D0230370AB
:10702000CE3B45708370C470307804F05DFB70BD5A
:10703000A83DFF1F70B5040006200D0004F064FB9E
:10704000011E0AD0D0230370CD3B8370054B4470E2
:107050001B688580187804F047FB002C01D0FFF7EF
:1070600067FF70BDF45EFF1FF8B5264F06003B6852
:107070000D001124002B05D10522234B1B78134250
:1070800002D112242000F8BD204A10241268002AE0
:10709000F8D01278002AF5D0DB0719D52B789A1E84
:1070A000012A1AD80C2004F087FB1324386000282A
:1070B000E8D000230A22437029000670023004F051
:1070C0001BFDFFF75BFF041E0AD0FFF731FFD9E776
:1070D00000F012FB0028E1D1E4E7002BE2D0D0E77A
:1070E0000B4B1B78032BCDD11D20FFF72BFA094B3F
:1070F00018800028C6D0084B04211878074A04F0ED
:10710000D3FCBFE7F45EFF1FF15EFF1F105FFF1FA0
:10711000F05EFF1FEE5EFF1F1C5FFF1F60EA0000B6
:10712000F7B50193194B14001A78052306000F00D8
:1071300012201A4221D0012920D1154B1D68002DA3
:107140001BD002201F2C18D8002C02D0019B002B32
:1071500013D0104B1F221E706E1C0021300004F053
:1071600003FB01992200300004F0C6FC310020002E
:107170002C70002F06D004F017FBFEBD064B12202A
:107180001D68DCE704F0D8FAF7E7C046F15EFF1FA0
:10719000105FFF1FA83DFF1F0C5FFF1FF8B50F4ECC
:1071A00012243368002B17D01B780F3C834213D175
:1071B00000250B4F0221387804F0D6FC094B04213E
:1071C00038781D8004F0D0FC074B28001D80336800
:1071D0005C7004F081FC04002000F8BDF45EFF1F29
:1071E0001C5FFF1F085FFF1FEE5EFF1F70B50128C9
:1071F00023D11B4C2388002B03D01A4A1578002D6D
:1072000007D0194B1B68002B02D01878FFF7C6FF78
:1072100070BD3B2B02D93C3B2380F9E7134E022182
:10722000307804F0A1FCFA222388920002215A430C
:10723000307804F0B1F92580EAE70B4B1B68002B8E
:10724000E6D00B4B1B785B07E2D5084B0221187880
:1072500004F08AFC0022024B1A80FFF769FED7E790
:10726000085FFF1FEC5EFF1FF45EFF1F1C5FFF1F28
:10727000F15EFF1FF8B51E4D2868002803D004F00A
:1072800013FB00232B601B4E3068002803D004F052
:107290000BFB00233360184F05243B781800204077
:1072A000234221D0154800F02BFA3B78234213D01B
:1072B000202004F081FA2860002813D02022002129
:1072C00004F052FA202004F077FA041E306005D052
:1072D0002022002104F048FA002004E0286804F08D
:1072E000E3FA2C601320F8BD00F00AFAF4E7C04678
:1072F000105FFF1F0C5FFF1FF15EFF1F9C3DFF1F14
:1073000010B50A4C23681A1E0ED0002808D101308F
:10731000587004F0E1FB002805D02368002B02D050
:107320000021FFF787FE0122100010BDF45EFF1F51
:10733000F7B5274E050033680191181E21D05C78FF
:10734000244F012C30D1FFF7FFFD002825D020006D
:10735000FFF7F8F80400412814D91F4B02211878D0
:107360001E4A04F0A1FB1E4B3C3C1C8002223368E9
:107370005A703B78002B14D128000199FFF75AFE70
:107380000120FEBDFA2292004243002AEED0124BA9
:107390000221187804F000F9E8E7FFF7D3F80200BB
:1073A000F3E700233B70EBE73B78002BE8D10320A9
:1073B00004F0AAF9011E08D0D0230370CC3B45701D
:1073C00083703368187804F08FF9FFF7B1FDD7E7C1
:1073D000F45EFF1FEC5EFF1F1C5FFF1F60EA0000F2
:1073E000085FFF1F10B51749838802008B4220D029
:1073F00011D815498B4217D0144900205B1899B257
:10740000012907D8926811785A425341D8B2FFF740
:10741000F9FD012010BD0E4A00209B1807229BB2E7
:107420009A424041C0B2F5E783681878FFF768FFD9
:10743000F0E7836899785A78090218781143FFF7C2
:1074400077FFE7E70A20000006200000F8DFFFFFD3
:10745000AFDFFFFF014B18707047C046A93DFF1F0B
:1074600010B5064C207001F041FA207804F0ECFAD7
:107470000521207800F062FD10BDC0461C5FFF1F93
:107480000BB273B50D00002B00DBC4E0884B1878FD
:1074900004F0EAFA041E0ED00378912B0FD0A22B31
:1074A00000D1A1E0834B1878FF2852D0210004F0CE
:1074B0001BF900284DD180200002684076BD43783A
:1074C0000F2B76D013D8052B70D00E2BEAD18088E5
:1074D000794B98422BD8794B98421BD8784B9842DD
:1074E000E0D1A3681878591CFFF774F838E03E2BF8
:1074F000D8D18378032B74D06CD8012B6ED0022B9B
:10750000D0D1704B1B68002B23D05B68002B20D0A0
:1075100098471EE06C4BC0180C28C3D804F05CF9E7
:107520001DC2C2150BC20B0B0B3223C23C00674BB2
:10753000C0180728B6D8664B1B68002B09D01B68FB
:10754000002B06D0200098470AE0A3681878FFF7C0
:10755000C7F8200004F010FBADE7A068FFF762F861
:1075600000289FD0F5E7A3681B78002BF1D0554B7E
:107570001B68002BEDD01B68002BEAD0210055487A
:107580009847EDE74F4B1B68002BE2D01B68002BA0
:10759000DFD021005048F3E7504B1B68002BD8D0B8
:1075A0005B68002BD5D021004348E9E7FFF7EAF9F3
:1075B000CFE780884A4B984203D04A4B984200D08C
:1075C00070E7464B1B68002BC3D05B68002BC0D014
:1075D0002100D5E7153B012BBBD963E7FFF798FAEC
:1075E000B7E7FFF77DFAB4E73F4B1B78042B07D1D1
:1075F00000236A4613800179408800F0C5FCA8E7A3
:10760000364B1B68002BA4D05B68002BA1D0010077
:10761000364898479DE7012421420AD0294B1B6830
:10762000002B04D05B68002B01D00020984701207C
:1076300043E78B070AD5264B1B68002B04D05B68F9
:10764000002B01D020009847022036E704212800B3
:1076500008400D4200D131E7254E3388002B21D060
:10766000013B9BB23380002B1AD1FFF7DBF80028D7
:107670000AD0204B1C70164B1B68002B04D05B6893
:10768000002B01D020009847FFF7C6F8694601F0AB
:1076900001FD6846FEF7FEFF1D20FEF753FF308018
:1076A00004200AE7024B187804F05EFAF8E7C046B7
:1076B0001C5FFF1FA93DFF1F0E20000001200000DE
:1076C00009100000145FFF1FFEDFFFFFAFDFFFFFA9
:1076D000185FFF1F0C2000000B200000FC5EFF1F46
:1076E0000D20000013200000F15EFF1FFFFF0000CF
:1076F000EE5EFF1FEC5EFF1F10B501F09BF910BDA1
:10770000014B18607047C046185FFF1F0B880020B0
:10771000162B01D817230420014A13807047C04656
:10772000C65EFF1F00207047074A03001188814290
:1077300007D091880020994202D1013080001018B2
:1077400070470020FAE7C046245FFF1FF0B58F782E
:1077500006000D00C5B01E2F15D1FFF7E5FF051E71
:1077600003D10024200045B0F0BD00223B003100D1
:10777000C078009200F0B2FB0400A81C00F0D2FB1D
:10778000FF23EB70EEE7264B062403931B78FF2BB9
:10779000E8D0182FE6D87B08224A013BDB00029292
:1077A0009A589446002ADDD0029AD3185B68002BC1
:1077B000D8D00878002802D14B78012B02D10624BA
:1077C000122FCFD107AFAB88697800976446AA68BB
:1077D000A047041EC6D1AB78029A5B08013BDB00D0
:1077E000D318390030005B689847041E0BD1AB7882
:1077F000042BB6D0039A310010782200009700F0D5
:107800006DFB0400AEE76A78002AABD1AA7805A91F
:107810003B88087130000A704B80FEF747FBA0E7F9
:10782000AC3DFF1FA0BD00111D4B37B505009842B0
:107830000BD000290AD1FFF777FF002805D119489E
:10784000FFF772FF002800D0058037BD01291AD14B
:10785000FFF76AFF041EF8D001235B420380A37880
:10786000FF2BF2D0FE2B07D00023E07814220093E8
:1078700029001E3300F032FBA01C00F053FB012353
:107880005B426380E1E70229DFD1013901F0BEF8F4
:107890000028DAD12800FFF747FF041EDFD1D4E724
:1078A000FEFF0000FFFF0000022210B5074B52420E
:1078B0001A80074801325A809A80DA8000F07EFAF6
:1078C000044801F025F8002010BDC046245FFF1FCA
:1078D0004D770011297800110388F7B50400002BBB
:1078E00002D102252800FEBD4268022113782548F6
:1078F0005268FEF7A5FD00282ED0234F01253A88B7
:10790000002AEFD0802321885B0201259B1A99422F
:10791000E8DC0C2003F050FF061E31D03B882288A3
:107920009C4600231800019561469DB2491989B211
:10793000AA421BD8002801D062443A8000233000BC
:10794000082208C0210004F0D7F8104A1368002B61
:1079500013D100251660C5E76268022113780C4830
:107960005268FEF76DFD0028C7D1BAE760681D01B7
:107970004019418101330198D6E71A001B68E6E7F8
:107980001325AFE70EBE0011AA3DFF1F205FFF1FAA
:107990000CBE0011014B18707047C046AC3DFF1F74
:1079A00014230A0010B51A40194204D001221021F4
:1079B00001F048F810BD4B06F9D40120884340007F
:1079C000F8E710B514008B0604D50122102101F050
:1079D00039F810BD08230A001A40194202D14BB2EF
:1079E000002B0FDA102101F02DF8002808D0230019
:1079F000F2331B78002BECD0F1342378012BE8D143
:107A00000020E6E703208907FAD4E2E7F0B51F007B
:107A1000184B85B01C68019002910392002C27D16D
:107A2000200005B0F0BDA5683301ED186B89019AFF
:107A3000934211D3029A93420ED8002F04D10A9B8D
:107A4000002B10D12C00EBE73B002978039A6868E3
:107A5000FEF7F6FC0028F2D10136B6B2A388B34295
:107A6000E1D82468DAE7A3680A9A5B891380E9E71A
:107A70000026F3E7205FFF1F37B50C000A8849880E
:107A80000123914217D3002A15D0651D23792A00BE
:107A900002210A48FEF7D4FC102300280BD02379DA
:107AA0006188208800242A000094FFF7AFFF0A2392
:107AB000A04200D0230018003EBDC0460EBE0011FB
:107AC00013B50A0008884988012388420BD800288A
:107AD00009D00024137905320094FFF797FF0A2399
:107AE000A04200D02300180016BD13B50A00088874
:107AF0004988012388420BD8002809D00024137933
:107B000005320094FFF782FF0A23A04200D0230031
:107B1000180016BDF0B58BB003904A8808880E0097
:107B20000123824255D3002853D00023012704ACFF
:107B300023700022718813000092FFF767FF051E73
:107B40003ED02078002835D12B78022B18D16770D1
:107B50006A8983000130E31880005A806968022234
:107B6000201803F0C9FF23780133DBB22370042B04
:107B700019D93B006889013080B2002BD9D01FE0B1
:107B800002236370122358436A89231804305A80F1
:107B900069681022201803F0AFFF23780133DBB2AD
:107BA0002370002BE5D10C4A6B899B185A42534134
:107BB000DBB2DFE76378012BE4D12B78022BC7D04F
:107BC00022780A23002A04D021000398FEF798F9AE
:107BD000002318000BB0F0BD0100FFFF0F4BF0B504
:107BE00004001868002816D083685D89A54207D86C
:107BF0008288AE18B44203DA12019A18934201D176
:107C00000068EFE71E005F891036A74204D1002903
:107C100000D00D801800F0BD3300EFE7205FFF1F9C
:107C200070B505000C0008880021FFF7D7FF03009E
:107C30000120002B04D022002800197AFFF7C1FE92
:107C400070BDF7B50C00002501902300EE331B78C2
:107C5000AB4201D800200AE06B00E65A0021300058
:107C6000E718FFF7BBFF002802D126800130FEBDD8
:107C7000017A0198FFF794FE002802D03B88238008
:107C8000F5E70135EDB2E0E710B504000888002102
:107C9000FFF7A4FF03000120002B03D02000197A76
:107CA000FFF77EFE10BD0000054B1B68002B01D1C5
:107CB000180004E09A6852898242F6D19888704789
:107CC000205FFF1FF0B50E27002687B0039302AB9D
:107CD000FF183E8005001F4B40891400984207D0D2
:107CE0002B78013000976A6880B2FFF78FFE06009C
:107CF00002212B7818486A68FEF7A2FB00280FD0F3
:107D00006C892000FFF7D0FF002802D0013C041945
:107D1000A4B2039B002B00D01C80300007B0F0BD44
:107D200002212B780D486A68FEF78AFB0028E7D10C
:107D300002212B780A486A68FEF782FB002807D0E8
:107D4000002EDED03B88A342DBD17489013CDFE703
:107D50006C89DEE7FFFF00000EBE00110CBE0011B3
:107D60000ABE001110B50C00FFF7DEFC0300022074
:107D7000002B0AD0002C00D023609B781720FE2B0C
:107D800003D00138FF2B00D1002010BD73B50D00CA
:107D900001A904001600FFF7E5FF172805D0002E03
:107DA00004D129002000FEF727F976BD0122102119
:107DB000200000F047FE0028F3D0F6E7014B1860E2
:107DC0007047C046305FFF1F37B56B469D1D0100F1
:107DD00004000222280003F02FFC2B88B02B0ED1C8
:107DE0002379122B09D12300FA331B78012B06D1FA
:107DF0000121608800F0E0F801E01B2BF8D037BDCE
:107E000010B5054B0421187000F098F8FFF74CFDF1
:107E1000FEF770FB10BDC046345FFF1F0020F0B5B9
:107E20000BB20F0087B0834234DA274B187803F087
:107E30001BFE051E2BD00378A02B25D103AE3100ED
:107E4000FEF7E4F8041E0BD1B378DB0724D51F4BF3
:107E500006341B68002B03D0310068889847040063
:107E6000A868002801D003F05FFD002C08D1184A53
:107E7000039B1340174A934206D0B3781B2B03D0C1
:107E80000121688800F098F8280003F075FE802032
:107E90000002784007B0F0BD0F4B1B68002B10D0DC
:107EA000310068889847041EDAD07378002BD7D148
:107EB000B27801A90A704B800C716888FDF7F6FF53
:107EC000CEE70624F1E7C046345FFF1F2C5FFF1F9B
:107ED00000FFFF0000011200305FFF1FF7B50190A7
:107EE000FC200D0017001E0003F00EFC0400132000
:107EF000002C12D0B02320002370089BF42267705E
:107F0000658026710830002B08D0190003F0F4FDBD
:107F10002100019803F0E8FB0020FEBD089903F062
:107F200023FCF5E710B5041E06D00078FD2803D821
:107F300003F02AFCFF23237010BD00000A1F93B238
:107F400010B504000220032B05D882400020024B0C
:107F5000D1529B189C7010BD545FFF1F0B8870B5E9
:107F6000043B04000D000220032B0BD8012120004C
:107F700000F04CFD03001420002B03D0290020004A
:107F800000F0DEFB70BD000007B51300034A00924D
:107F90000A00012100F02CFC0EBDC046C581001175
:107FA00007B5019203220092024B0A00122100F051
:107FB00049FC0EBD4382001107B56B4601AA118032
:107FC0000449D88008780633012802D1190003F04B
:107FD00023FB07BD355FFF1F0C4B10B51870002346
:107FE000FF210B4A1380138193819380094A5380A8
:107FF0001370517293819372D174D3821375517738
:1080000003F01AFD00F0FCF910BDC046645FFF1FCD
:10801000545FFF1F365FFF1FF0B58DB06B46002029
:1080200003910C229B5E834200DBB0E05D4B18782D
:1080300003F01AFD051E00D1A4E00378902B00D0B8
:108040009DE006AF01004688380000F013FA796819
:108050000400002900D19CE03B88052B6ED13B89B0
:10806000032B1CD905AC200000F0A2F86288172A67
:1080700061D83989131D994231D179682378043147
:108080000291D90738D5607800F08EF9071E06D026
:10809000002303712378012B08D0132B23D0A86869
:1080A000002800D178E003F03FFC75E06288029977
:1080B00009A800F0A6F80290380000F08BF909AA90
:1080C0002378387A0192002231000092029A00F05F
:1080D00012F9380000F064F9029B002BDFD0300069
:1080E00000F080F9DBE70378032BD8D1628802998E
:1080F00009A800F0D6F8DEE7122B13D1029909A8DF
:1081000000F0B5F8021EEAD127498B88002BC6D0B3
:10811000887909A92378019161780091310000F0F4
:10812000EAF8BCE7002302AA93833000617809AA29
:10813000FFF72AFFB3E71D4B0993F6E7042B02D0A4
:108140009A1F012AABD8184A043B9B00995A002970
:10815000A5D0D218907831003A0000F0AEF800288F
:108160009DD13B88042B03D001213000FFF724FF71
:10817000012C04D1A868002801D003F0D5FB280009
:1081800003F0FAFC8020039B0002434018000DB06E
:10819000F0BD012800D182E701213000FFF70CFF7C
:1081A000EDE7C046645FFF1F545FFF1F010017002B
:1081B0000B7803704B784370CB788A781B0213439B
:1081C000438070470A88030002700A88120A4270CE
:1081D0000A88012A06D14A8882704A88120AC27027
:1081E0000420704702208242FBD14A8804309A70F2
:1081F0004A88120ADA708A881A718A88120A5A71B1
:10820000EFE710B50400012082420CD94B780A78C0
:108210001B0213432380834206D1CB788A781B024A
:1082200013436380002010BD022BFBD1CB788A78EA
:108230001B02134363804B790A791B021343A3800B
:10824000F0E70B8803700B881B0A43704B88837020
:108250004B881B0AC3708B8803718B881B0A437180
:10826000CB888371CB881B0AC37108207047030039
:108270000120082A14D14A780878120202431A8091
:10828000CA788878120202435A804A790879120221
:1082900002439A80CA798879120202430020DA8068
:1082A000704710B504000120022A05D100204B7848
:1082B0000A781B021343238010BDF8B50600102076
:1082C0000F00150003F020FA04000120002C0ED04E
:1082D000A0230C22290023806780201D002D07D0B9
:1082E00003F00AFC2100300003F0FEF90020F8BD85
:1082F00003F03AFAF6E7F7B51E00009008AB142039
:1083000017001D78019103F0FFF9041E12D0A2237B
:108310000370019B47704380099B057146710C22D5
:108320000830002B07D0190003F0E6FB210000986D
:1083300003F0DAF9F7BD099903F016FAF6E737B555
:10834000041E0FD04388002B0CD00025C1881323B6
:10835000007A172201950095FFF7CDFFFF23658076
:108360006372257037BD000010B50C4904004A88BF
:10837000002A09D08B89002B05D00020CB8A02224D
:10838000834201D010BD012213000A204343002084
:108390004032C854C81842800472F3E7365FFF1FAA
:1083A0000023438003707047094B00211A0010B569
:1083B0005C88002C06D01C79844203D10A234B43ED
:1083C000D01810BD01310A330329F1D10020F8E79C
:1083D000365FFF1F10B50400407A03F0D5F9FF2384
:1083E000637210BD7047043010B580B203F0D4FB47
:1083F000002803D00421494203F0A6FA10BD000072
:1084000070B50025104CA0682580A581A580A842E4
:1084100002D003F089FAA56000250C4C0C4B606D6E
:108420001D80230058331D70A84202D003F07CFA4F
:10843000656500256068002801D003F075FA0135F4
:1084400008340A2DF6D170BDFC5FFF1FA05FFF1F2F
:10845000F05FFF1F70B5041E09D1054D2880A8816B
:10846000A880A868002802D003F05EFAAC6070BD56
:10847000FC5FFF1FF0B54B8885B00193002343607C
:108480000A7905000F00022A00D07BE0CA88032A7F
:1084900017D98B685E7819783602DC78D8790E4364
:1084A00099781B7A24021B020C43034353495BBA9D
:1084B0000B80331D93421ED1042C04D0631F022B6A
:1084C0000ED9012015E0019A4D4B1201D35A002B11
:1084D00006D00198FFF7BEFF4A4A136901331361C2
:1084E0000421B8682E812C80494203F02DFA68607F
:1084F000002005B0F0BD434D042C06D0631F022BB5
:108500000FD9EB680133EB60DBE7019A3C4B1201BA
:10851000D35A002B05D00198FFF79CFF2B6901333C
:108520002B61374B30000293019B029A1B01019390
:10853000002301998C468B52130063449C80039363
:108540009E81FFF750FF039B041E986016D0042104
:10855000B868494203F0F8F9FA880100043A2000AB
:1085600003F0CAFA0199029AFB888A5A043B9B18C5
:10857000029A8B522B6801332B60A2E7AB6901335F
:10858000AB619EE71E4B0293019B1E01029BF35AB7
:10859000002B2DD002998C19A068002828D0012A20
:1085A00026D1FA889B189BB27352A189994217D39E
:1085B0009B1AC018B96803F09FFA029BA289F35A6C
:1085C000934200D07DE700222B81A3882B80A368F3
:1085D0006B60029BF2520B4A53680133536070E7A1
:1085E000084A9368013393600198FFF733FF68E707
:1085F000044A536901335361F6E7C046665FFF1FC3
:10860000FC5FFF1F6C5FFF1F70B5051E15D10B4C83
:108610000B4B1880230058331870606D002802D06F
:1086200003F082F96565250050356068002801D0A7
:1086300003F07AF90834AC42F7D170BDA05FFF1F98
:10864000F05FFF1FF0B51700A12285B092000193E3
:108650004243394B06001B680C009B18D933FF338B
:108660001D78FDF741FF0430854204DD3000FDF741
:108670003BFF0430C5B2BD4207D33A0000213000B1
:10868000019B03F011F805B0F0BD2900380003F09C
:10869000BBF92300C6B250331E700393019B29001F
:1086A0006365380003F078F8CBB20293002B02D058
:1086B000039B01361E7000262300503303931B7862
:1086C000B34204D8606D002831D10020DBE7029A64
:1086D0002800002A04D0013B1000B34200D028003B
:1086E000F700E719387002F0D7FF786000280ED045
:1086F0003A78019903F000FA019A3B780136D318D1
:108700000E4A0193D369F6B20133D361D4E7039BD8
:1087100018706065A74205D1084A1320D36A013357
:10872000D362B0E7606803F0FFF80834F2E703F0C3
:10873000FBF800236365C8E73409FF1F6C5FFF1F68
:10874000F7B50D0007000421686803F0FDF82B89D8
:10875000040003702B891B0A43702B8883702B88BD
:108760001B0AC3702E8902250436F6B2F42E15D8E2
:108770001B4B9F4214D10C2002F0C6FF1135011E85
:108780000CD0902303708E3B0371043B4380154B48
:108790008460C680187802F0A7FF00252800FEBD7F
:1087A0005C237B43104AD3180093583301931B7802
:1087B000002B0FD10300320038000099FFF742FF71
:1087C000019B05001B78002BE8D13800009903F0CD
:1087D0005BF8E3E7054A0725536A01335362DDE797
:1087E000FEFF0000645FFF1FA05FFF1F6C5FFF1FA5
:1087F000F0B587B0009017200F0016000193FFF727
:10880000F2FD1325041E19D00C98031E02D0019905
:10881000201D9847030AE370052302AAA0700430C4
:10882000908127700098667003A993800494FFF7E5
:1088300087FF051E02D0200003F076F8280007B05D
:10884000F0BD0000F0B587B01F000CAB1B780391A2
:10885000059301210DAB06001C78049200F0D6F8B8
:108860001425002821D02000FFF77EFD0135041ECD
:108870001BD01149059B0A7803700132D2B2131E36
:10888000C68001D101231A000B7022713000049BB5
:1088900003990097FFF7ACFF051E09D123002100C3
:1088A0000648074A093303F07FF8280007B0F0BDF7
:1088B000002363802370F8E7685FFF1F3F83001188
:1088C00030750000F8B505000E00064C064F236811
:1088D000002B02D03100280098470434BC42F6D166
:1088E000F8BDC0460C60FF1F2060FF1F0123064A31
:1088F0005B425380002313715362044A1360536038
:108900009360D360136170472060FF1F0C60FF1FEE
:108910000200002310B506499C000859002801D127
:10892000625010BD0133052BF6D11320F9E7C04684
:108930000C60FF1F034A5388181A434258414042B3
:10894000104070472060FF1FF0B585B002930AAB5E
:108950001F780CAB1B88009008000E000192039357
:10896000FFF7E8FF05001120002D1BD10E48FFF78F
:10897000E1FF04001520002C14D006220B99A771EA
:10898000E01D03F0B9F8019B30002371029B290020
:108990006371009B66802370039B6562E381FFF730
:1089A00091FF280005B0F0BDFFFF000010B5FFF7F4
:1089B000C1FF04000220002C12D060880121FFF7C3
:1089C00081FF606A002801D002F06EFF282200219A
:1089D000200002F0C9FE012300205B426380207169
:1089E00010BD000030B5074A074C558801001378C8
:1089F0000020A54204D05B1A59424B415842104016
:108A000030BDC0462060FF1FFFFF0000084A10B5C0
:108A100001230C00904208D0FFF78CFF031E04D006
:108A2000037923405A1E9341DBB2180010BDC046A3
:108A3000FEFF0000024B1879431E9841C0B27047F8
:108A40002060FF1F70B504000D001600FFF772FFD5
:108A5000002804D10D4B9C4200D0143070BD416AF7
:108A600003790520002907D012221A40102A02D1CA
:108A70000520002EF2D10F20DB06EFD5897E0C20D9
:108A8000A9428941494249420840E7E7FEFF000008
:108A9000030010B5002800D110BD0348034A4188E7
:108AA0009142F9D09847F7E72060FF1FFFFF0000D1
:108AB000002330B5C45CCD5C6C40D4540133102B22
:108AC000F8D130BD0F23002210B5C45C64002243EE
:108AD000CA54C25CD209013BF7D210BD02000100AA
:108AE00010B52032103102F0AFFE10BDF0B58BB0E2
:108AF0000390102005931700049102F05DFE009092
:108B0000102002F059FE009B13240190002B05D089
:108B100000280CD11324009802F0C6FE019B002B04
:108B200002D0180002F0C0FE20000BB0F0BD1020F3
:108B300002F042FE0600102002F03EFE1324050063
:108B4000002E00D1AEE0002819D01022002102F042
:108B50000BFE32002900039802F076FE041E0ED1AF
:108B600033787F2B51D830000099FFF7ABFF009B83
:108B70001B787F2B53D801990098FFF7A3FF300093
:108B800002F092FE002D02D0280002F08DFE002C93
:108B9000C1D1102002F010FE0600102002F00CFEE1
:108BA0000290002E7CD0002878D03A000F322300AB
:108BB0000125121105D00F333B4015B25A425341E3
:108BC0001BB26A1E1201002B33D0049BD2B298183C
:108BD0000099029AFFF76CFF013D1022002130003E
:108BE00002F0C2FDADB2049F2D017D19AF4242D00B
:108BF000002C33D0300002F057FE029B002B00D136
:108C000089E7180002F050FE85E729003000FFF7E1
:108C100059FF28002549009AFFF74AFFA7E72900D6
:108C20000098FFF74FFF28002049019AFFF740FF07
:108C3000A5E70F210F4004998A18D9B28F4208D9AD
:108C4000D15C06A819540133102BF6D1029A019970
:108C5000C0E7791A48424141C901F2E739003000C2
:108C600006AAFFF725FF3200039806A902F0ECFDE3
:108C700010370400BAE7002CBCD13000029906AAD4
:108C8000FFF716FF320006A9039802F0DDFD082267
:108C900004003100059802F02FFFABE71324A9E789
:108CA0001324AAE7002800D06EE733E714BE0011B2
:108CB000F0B58BB00F0016000225009000283FD0C1
:108CC000002A3DD00B1DDBB21800029302F074FDA8
:108CD0001135041E34D0FDF747FD05003A00009918
:108CE000201D02F0F9FDEBB20393E3702B0CDBB215
:108CF0002F0A00936370FFB22B0E2370A7700193AD
:108D0000FDF72CFD1022010006A802F0E5FD210070
:108D1000029A04AB06A8FFF7E9FE051E0DD1039BDE
:108D200008223370009B04A9B370019B7770F37025
:108D3000301D02F0D1FDFDF71DFD200002F0B4FD55
:108D400028000BB0F0BDF0B58FB00D00149E03905D
:108D500004920593002A03D1022420000FB0F0BD35
:108D6000002EF9D00398FFF7E5FD1424071EF4D078
:108D70007278337812021A43B3781B041343F278E3
:108D800012061A43036A0192934201D30133E3D1DD
:108D9000002D03D03B7901249B07DED5082200215A
:108DA00006A802F0E1FC059B13240433DBB2180093
:108DB000029302F001FD051ECFD0059A04990430FC
:108DC00002F08AFD04223100280002F085FD3900FE
:108DD000102210310AA802F07FFD2900029A06AB8A
:108DE0000AA8FFF783FE041E0FD1082206A908A8CF
:108DF00002F072FD0822311D08A802F06DFC012866
:108E000007D101990398FDF7C9FC280002F04CFD39
:108E1000A3E70124F9E7000070B51C4C05002368A6
:108E2000181E10D0002D14D11A78002A0CD1981CCD
:108E3000083202F061FE02F017FC0135002808D16B
:108E400023681D70012070BD0A331800082202F04B
:108E500053FE2368002BF5D0122002F055FC061EAD
:108E60000DD0C123216803704570023110220230F9
:108E700002F042FE23683100587802F035FC206889
:108E800002F012FD00232360DCE7C0464860FF1FAC
:108E9000F8B504002020FDF755FB0D4EA700BB5987
:108EA0000500002B0DD000280BD0D878FF2809D161
:108EB00008492A000C55F35907480333611802F09A
:108EC00073FDF8BD290002F077FD0028F0D1F8E726
:108ED0006460FF1F4C60FF1FE9A0001170B5064DD4
:108EE00084006359002B05D0D87802F04DFCFF2296
:108EF0006359DA7070BDC0466460FF1F70B506002C
:108F00008CB00C00150000213022684602F02CFCC9
:108F100031001022684602F0DFFC1D2021000322F0
:108F2000684402F0D9FC6846FFF7D8FD2D21040003
:108F300003222800694402F0CFFC20000CB070BD71
:108F4000F0B50700160097B001931CAB1D783022D6
:108F50001EAB00910AA800211C7802F005FC10222B
:108F600039000AA802F0B8FC1022002102A802F081
:108F7000FBFB0722310002A802F0AEFC072202AB85
:108F80009818631E9C41019902F0A6FC02AB9C73E9
:108F90002B005A1E934102AAD3730021102206A867
:108FA00002F0E2FB06221D9907A802F095FC1A20A8
:108FB00002ABC01806221F9902F08EFC1022009905
:108FC0000EA802F089FC102202AB0EA908781C78CA
:108FD000013A6040D2B2087001330131002AF5D164
:108FE0000AA8FFF77BFD102212A904000EA802F0C8
:108FF00083FD102206AB0EA908781D78013A68405F
:10900000D2B2087001330131002AF5D10AA8FFF766
:1090100065FD044310222098E4B212A902F05CFC22
:10902000200017B0F0BD70B50E0014008CB0010028
:10903000102268461D0002F04FFC3100082204A8EF
:1090400002F04AFC2100082206A802F045FC68460E
:10905000FFF744FD04001022280008A902F03CFCA0
:1090600020000CB070BDF8B506000D0000243719C3
:10907000AC4200D3F8BD02F06FFC030A3B70631CE6
:10908000DBB201379D4203D90234F054E4B2EEE77B
:109090001C00EDE773B506000C000225002819D06E
:1090A000002917D0032101A8FFF7DDFF6B469A794D
:1090B0003F231A40013313436A463000937101A9DC
:1090C0002200FFF71BFF051E04D10322E01C01A9AB
:1090D00002F012FD280076BD03785807DA08C00FA9
:1090E000D20080009B0710439B0F1843C0B270470B
:1090F00007230B40C908C9000B43037070470000E9
:1091000070B50400FFF7EAFE134DA4006359002B6D
:1091100021D0186A002801D002F0C6FB2B59986EA6
:10912000002801D002F0C0FB2B59D86E002801D0D6
:1091300002F0BAFB2B59186F002801D002F0B4FBE3
:109140002B59586F002801D002F0AEFB285902F0CD
:10915000ABFB00232B5170BD6460FF1F0E4B8000E2
:10916000C35870B50C00002B0FD09D68002D0CD09B
:109170002B78201D0B706B784B70A97CFFF7B8FF24
:109180002B7E23726B69E36070BD102200212000EA
:1091900002F0EAFAF8E7C0466460FF1F014B18606E
:1091A0007047C0466060FF1F074A03008000825876
:1091B00010B5002A06D0D088984203D1012901D1E8
:1091C000FFF79EFF10BDC0466460FF1FF0B5264E3E
:1091D00095B087000B93BB590500099112200A92A4
:1091E000002B31D0D888FFF7A5FB04001420002CF9
:1091F0002AD0280010A9FFF7B1FFBB591E781D6ABD
:10920000002E23D00895FDF7EFFA07000020FDF7A8
:10921000F1FA0790A379E61D069310AD0CA9089802
:1092200000F0E2FA0EA9280000F0D7FA0B9B0A9989
:109230000493069B09980293079B0396019300975A
:109240000EAB0CAAFFF77CFE15B0F0BDFDF7CCFA13
:1092500006903000FDF7CEFAE31DA779079310AB17
:1092600006000893DAE7C0466460FF1F30B50C4C77
:1092700085002A59030085B00120002A0ED018006D
:109280006946FFF76BFF2B591A78D888054B002ADF
:1092900000D1054B6A46072100F0D9FB05B030BD6F
:1092A0006460FF1FDB970011E997001130B5094C8E
:1092B0008500295985B010226846253102F01CFC32
:1092C0002A591121044BD0886A4600F0C0FB05B032
:1092D00030BDC0466460FF1F8598001130B5094C51
:1092E0008500295985B010226846353102F004FC0A
:1092F0002A591121044BD0886A4600F0A8FB05B01A
:1093000030BDC0466460FF1FC3980011F7B54D4FD4
:1093100086001020F4590D0002F04EFAF359206235
:10932000186A132200286CD0033A29009C6802F0C6
:10933000E3FBF3591A780192002A58D11E6A227D64
:10934000317B944651400122019F114201D1674671
:109350001740217D914339432175377B4F40BC46EF
:1093600060460027800701D44F08174001210220E2
:109370008F40227D82433A432275377B5740BC465B
:1093800060460027400701D497080F400420227D43
:10939000BF0082433A432275627D002794466046AF
:1093A000727B42400A4201D167460F400121627D33
:1093B0008A433A436275777B5740BC466046002734
:1093C000800701D457080F400220627D7F0082434E
:1093D00017436775767B00227E40760701D4BA0872
:1093E0000A400426617D9200B1430A4362756A789F
:1093F000002A08D06278002A05D005220533DA77E2
:1094000000221000FEBD04222979114205D1A17C61
:10941000114202D10533033AF1E7019A21782C7801
:10942000002A02D10A002100140018220429E8D8D9
:10943000042CE6D805206043034A05331218525C19
:10944000DDE7C0466460FF1F24BE001110B50A00AE
:109450001121024B00F0FBFA10BDC0461F9900110C
:109460000B0030B587B001AD2B806B4604001100B6
:10947000981D082202F040FB2A000B212000024B1D
:1094800000F0E5FA07B030BD4799001110B50A00A9
:109490001121024B00F0DBFA10BDC0469B99001170
:1094A00013B50B0011006A4613706B4604000622C8
:1094B000581C02F021FB6A4608212000014B00F0F5
:1094C000C6FA13BDBB99001110B50A001121024B59
:1094D00000F0BDFA10BDC0460B9A00117FB5050023
:1094E0000B4BAA00D4580800002C0FD0666F237FC6
:1094F000E28821780396266F0296E66E0196A46EA6
:109500000094FDF709FC2800FFF7FAFD7FBDC04677
:109510006460FF1F10B51721FFF7E0FF10BD0000CA
:1095200070B50A000D00064B0221040000F08FFA0E
:10953000060029782000FFF7D1FF300070BDC0463B
:10954000EB98001170B586B000236A4613708368EB
:1095500004001D78681E0A2859D801A902F07CF879
:10956000060633373B3F43474B4F5300180000F08C
:1095700042F9062312284BD000281BD16088FFF740
:10958000D9F90823002813D04279002A47D1264B65
:109590001A78072312070BD5244B1A680723002AD1
:1095A00006D01668002E03D0290001AAB047030098
:1095B0006A4613706B461B786088002B2AD1FFF730
:1095C00067FC06B070BD180000F06CF9D4E7180015
:1095D00000F087F9D0E7180000F093F9CCE7180005
:1095E00000F0ADF9C8E7180000F0C3F9C4E71800AF
:1095F00000F0F6F9C0E7180000F0F6F9BCE7180033
:1096000000F013FAB8E7180000F013FAB4E70723E4
:109610006A46137069466088FFF782FFD1E7052329
:10962000012AC5D1024BB8E7F15EFF1F5C60FF1F46
:109630006060FF1FF8B52C4F8600F35904000D0041
:10964000002B40D0DA8882423DD15A78062A33D1A5
:109650001A78002A2ED0012099681A6A097D0142E1
:1096600006D0157B054203D007225A700120F8BDB1
:109670000220014204D0157B054201D00922F4E703
:109680000420014204D0127B024201D00B22ECE7FD
:10969000164B1B68002BE9D05B68002BE6D020003E
:1096A0009847BB5900215B78122BDFD12000FFF7D0
:1096B00015FFDBE70E4BECE7112A04D1002900D09F
:1096C00032252900F2E7002D08D12000FFF732F9FA
:1096D000002803D0102302791343037121002800CE
:1096E000FDF798FAC2E7C0466460FF1F5C60FF1F89
:1096F0006060FF1F70B50E4E8500AB590400002B53
:1097000013D01B78002B11D10A4B1B68002B04D0FF
:109710005B68002B01D02000984773595B78122BAF
:1097200003D100212000FFF7D9FE70BD024BECE70A
:109730006460FF1F6060FF1F5C60FF1F094B8000BB
:10974000C3581020002B0CD01A6A002A09D09B683D
:10975000002B06D0127A1B7E101C9A4200D9181CCE
:10976000C0B270476460FF1F70B503000D001400A5
:109770000220002A30D000292ED013700B78081D4B
:1097800053704B789370FFF7A7FCE0700120022123
:109790002B7A23716B7B034063716A7B0A4013430E
:1097A000042263716E7B1640334363716E7BF6084F
:1097B000F600334363712B7B0340A371287B014088
:1097C00000200B43A371297B0A401343A3712A7B1A
:1097D000D208D2001343A37170BD10B50A00010076
:1097E0000120FFF7C1FF10BD10B50A0001000220E3
:1097F000FFF7BAFF10BD70B506000C000220002E66
:1098000030D000292ED07378201D0B70B3784B70A8
:10981000F178FFF76DFC01223579257271794B10D3
:10982000080013409340104003438810104080000C
:10983000C9080343C9000B436373B1794B10080097
:109840001340934010400343881002409200C9081F
:109850001343C9000B4321202373FCF773FE854299
:1098600001D2122070BD2220257AFCF76BFE8542C2
:10987000F7D823781820042BF4D86378012BF1D87B
:109880000020EFE7030010B50220002909D0002BCB
:1098900007D00322481C0A7019000D3202F02CF97F
:1098A000002010BD03000222080010B5002B06D0D6
:1098B000002904D00E32591C02F01EF900221000BB
:1098C00010BD030010B50220002909D0002B07D0DD
:1098D0000422481C0A7019000C3202F00DF9002015
:1098E00010BD10B5FFF7DEFF10BD030002200029F8
:1098F00006D0002B04D0052200200A701B784B7084
:10990000704703000220002B08D0002906D05B78A6
:1099100000200B70013B082B00D918307047030062
:1099200010B50220002909D0002B07D00622481CC0
:109930000A7019000A3202F0DFF8002010BD10B5DD
:10994000FFF7B0FF10BD02000B00022010B5002988
:109950000ED0002A0CD00721197011885970118877
:10996000090A997011180822D81C02F0C5F80020C5
:1099700010BD03000A00022010B5002B0CD00029F6
:109980000AD099785878090201431180901CD91C9B
:10999000082202F0B1F8002010BD030010B502202B
:1099A000002909D0002B07D00822481C0A70190092
:1099B000921802F0A1F8002010BD02000B00022056
:1099C00010B500290BD0002A09D00921197011788F
:1099D00018185970511C062202F08EF8002010BD94
:1099E00010B5FFF75FFF10BD02000B00022010B59D
:1099F000002A09D0002907D05178197011180622C1
:109A0000581C02F079F8002010BD030010B50220A8
:109A1000002909D0002B07D00A22481C0A7019001F
:109A2000063202F069F8002010BD10B5FFF73AFFCA
:109A300010BD02000B00022010B5002A06D000293C
:109A400004D018005178FFF753FB002010BDF0B58B
:109A500085B017001E006A460623050008009181A4
:109A60009380FEF7C0FC1324011E02900CD0380036
:109A7000B047041E05D1280001A9FEF76FFA041EA5
:109A800002D0029801F050FF2800FFF701FA2000F1
:109A900005B0F0BDF0B504008BB0019115000021B8
:109AA000102202A801F060FE334EA700B85900282A
:109AB0003CD0C388A34239D10378002B36D14278F9
:109AC000062A18D102000100553235310C3006ABA0
:109AD000FFF7A9FA002829D12000FFF72FFE020086
:109AE00006A902A802F008F8200002A901F02CFE45
:109AF00001200BB0F0BD816E002917D00B8A112A0E
:109B000028D19D420ED101981231093A01F0E4FDAD
:109B1000012807D1BB5920009D6EFFF70FFE2900D9
:109B20000200DEE732212000FFF7D8FC2000FEF71C
:109B300001FF061E1BD0416A002918D00B8AAB42D8
:109B400015D108220198123101F0C6FD01280ED16D
:109B5000716A0AE09D42E9D108220198123101F0B0
:109B6000BBFD0128E2D1BB59996E8A7EB9E720007E
:109B700002F022F8BCE7C0466460FF1FF0B56B4DF1
:109B800087007E5985B0337802900393002B00D074
:109B900087E0B368346A01937078062817D10122F0
:109BA0001B7D134202D0217B114218D102221342A5
:109BB00002D0217B114251D10422134203D0237BD6
:109BC000134200D08BE0019B5A7DEB5991E007389E
:109BD0000428F8D801F040FD032E42678300B36EDD
:109BE000002B03D11C2001F0E7FDB066EB599C6E01
:109BF000002C1CD010220021200001F0B5FD02989D
:109C0000FFF79CFD01002000FFF72DFA01F0A4FEF4
:109C10002082200008211230FFF725FA0298FFF772
:109C20008DFDA076EB592100D888FFF70FFC0822A4
:109C3000EB591CE0B36E002B05D01A00198AF0888E
:109C40001232FFF70DFC0222019B197DEB591142E4
:109C50003DD0207B10423AD0073208E0F488FCF770
:109C6000DBFD01002000FFF711FC0A22EB595A70BE
:109C7000029B9C002A595378073B042B11D8D088AB
:109C8000FEF758FE00284ED0C3895A08D21828493A
:109C9000029B0298CB542B5941180433254801F0FC
:109CA00083FE05B0F0BDFCF79FFD03000120834259
:109CB00001D100200393EB59DE88FCF79BFD03994B
:109CC00002003000FFF7ECFB019AEB59117D0422F2
:109CD00011420CD0217B114209D00B22C7E7F68834
:109CE000FCF73CFD01003000FFF7EEFB6BE7019A4B
:109CF000527D01210A4204D0607B084201D00C222F
:109D0000B5E702210A4204D0607B084201D00E224E
:109D1000ADE704210A4204D0627B0A4201D010223E
:109D2000A5E71222A3E7FA225200B0E76460FF1F02
:109D30006860FF1FF3A0001110B5064B1A780423CA
:109D4000100018401A4200D00348FFF727FA0020FD
:109D500010BDC046F15EFF1FB03DFF1F70B504008F
:109D6000FFF7D4FA051E43D12000FFF77FFA234EF8
:109D7000A400A0598268937CDB0708D50321036AFD
:109D80001B790B40012B02D1017F0B430377431D4D
:109D9000D97F8B1E022B0DD8022900D00121C0884B
:109DA000FCF790FF042133591A7F59700A431A7740
:109DB000280070BD01290CD102231022437000211C
:109DC0000C3001F0D1FC305910213530FFF74BF940
:109DD000EEE70529ECD10223D118437010220C3094
:109DE00001F08AFE04233259117F0B431377EAE70F
:109DF00008251828DCD1053DDAE7C0466460FF1F5E
:109E0000F0B58BB0059143887E4F9E00F459150044
:109E10000493002C15D1012902D000200BB0F0BD15
:109E2000101D57781678FFF757F9EB683200029348
:109E30002B7A0499019300903B002000FCF70CFF63
:109E4000EBE7E388049A934201D00820E6E7237801
:109E5000012B00D1D4E0059B581E092800D9CFE082
:109E600001F0FAFB05CE0A29CC506C859AB2290084
:109E70000498FFF773FFD1E7200029001022453036
:109E800001F03AFEB9594B78042B02D1013B4B70DB
:109E9000C3E70B000A00253335320C310498FFF775
:109EA00095F90498FFF702FA0522431E9841BB5921
:109EB000C0005A70B2E7200029001022553001F08E
:109EC0001BFE049B4F4C9D00295904980A0006ABC9
:109ED00055320C31FFF77AF929591022453106A87D
:109EE00001F0FAFB012808D10498FFF7F7F9059073
:109EF000002804D106222B595A7005988EE70823B2
:109F00000593FAE763780C2B7AD1E36E002B03D12B
:109F10001C2001F051FCE066BB59D86E00286FD0C0
:109F20001022290001F0E8FDBB590498DC6EFFF710
:109F300005FC0D22A076BB595A706EE7E06E002832
:109F40005ED063780D2B5BD12B8808220382A91C7D
:109F5000123001F0D1FDBB599A68517D02221142A5
:109F600026D0186A407B104222D00C32E4E7637896
:109F70000E2B45D1236F002B03D1162001F01CFCC2
:109F80002067BB59186F002803D01022290001F068
:109F9000B3FD0F22BB59CFE763780F2B30D1206F71
:109FA0000622691C103001F0A7FDBB599A68517D4B
:109FB0000422114203D0196A497B1142D5D10021F4
:109FC0000498FFF78BFA28E7636F002B0DD0BB597D
:109FD000586F0028F3D01022290001F08DFD0122D6
:109FE000BB5952425B6F1A61E9E7142001F0E4FBB0
:109FF000BB5960675B6F002BE9D126E72978DFE763
:10A0000007200BE76460FF1F10B5064C207001F0BD
:10A0100003FD06212078FDF791FF0348FEF778FC49
:10A0200010BDC0467760FF1FA991001100200BB240
:10A0300070B50D00834216DA264B187801F014FD36
:10A04000041E0DD00378922B0ED0A02B37D0224BBC
:10A050001878FF283AD0210001F046FB002835D1BE
:10A0600080200002684070BD43780E2B0BD03E2B41
:10A07000EDD18378052B12D0082BE8D18179808827
:10A08000FFF7D8FA08E0154B82889A42DFD183683F
:10A090001878591CFEF7C0FE002817D1D7E7104BDF
:10A0A0001B785B0712D50F4B1B68002B0ED09B68EB
:10A0B000002B0BD0C289811D80889847ECE7FFF701
:10A0C00041FAA068002801D001F02EFC200001F028
:10A0D00053FDC5E77760FF1FA93DFF1F1820000053
:10A0E000F15EFF1F6060FF1F10B50078FFF712FAE6
:10A0F00010BD10B50078FFF7FDFA10BD0C234343E7
:10A10000084A10B59B185A68002A03D0012901D1CA
:10A11000904710BD9B68002BFBD00029F9D19847D0
:10A12000F7E7C0469460FF1F01238340094A10B53A
:10A13000946B1C439463506B98435063D46B200022
:10A140009843012901D120001843D063116B0B43C0
:10A15000136310BD00800040F0B500240127154BAB
:10A1600085B0DA6B144E03921A6C0192DA64019B8B
:10A17000E3403B4217D0039DE5403D400295E5B2E8
:10A1800002992800FFF7BAFF316A736A002908D0E4
:10A190003900002B01D0029979402800FFF7C4FF55
:10A1A00001E0002BF9D101340C36172CDFD105B0BA
:10A1B000F0BDC046008000407860FF1F064B0121C3
:10A1C0005A68C2400A4204D01B68C34018000840C5
:10A1D00070471B6DF9E7C046008000400122064B26
:10A1E0008240002903D0D9680A43DA607047D968F1
:10A1F0009143D960FAE7C0460038004030B50324E7
:10A2000044430F4BE25C1B199C785D7801232D1BA6
:10A210000135AB40013BA340A140DB430C001228B9
:10A2200007D808499200521811681940214311605B
:10A2300030BD054A11680B4023431360F8E7C04660
:10A240006BBE001108F0004014F00040C21F70B552
:10A25000D4B20623092C0BD80125084C95400029BF
:10A2600008D00021FFF7CAFF23682B432360002397
:10A27000180070BD2368AB43F8E7C04600380040C3
:10A28000214BF0B51B185B78022B21D103244443EA
:10A290001E4A1F4EA35C12199478012215008540B6
:10A2A000B76B013CE4B23D43A240B563194C1228A0
:10A2B00015D89B0000290CD117495B1899680A43EF
:10A2C0009A600123205C154A834011680B43136098
:10A2D000F0BD11495B18996891439960F1E70E4B05
:10A2E00000290DD159690A435A61225C1328E8D02C
:10A2F0000123203A93400A49086803430B60E7E7CB
:10A30000596991435961F0E77860FF1F6BBE0011F6
:10A3100000800040B0BE001100F00040A0F00040FE
:10A32000A4F00040F8B500241B4E1C4D1C4B1B5DD7
:10A33000012B1FD1194A9269E2401A420BD0012227
:10A34000B25693402200143AD2B2022A09D81549D3
:10A350004A6913434B61013402360C35172CE5D1A1
:10A36000F8BD0022B2560F499200521891680B4373
:10A370009360F0E7022BEED1E7B23800FFF71EFF43
:10A3800001235840C1B23800FFF77AFF3800FFF7C9
:10A3900015FF6877DFE7C0463DBE00117860FF1FFC
:10A3A0007960FF1F00F00040012202388240054B17
:10A3B000002903D059690A435A617047596991438A
:10A3C0005961FAE700380040F8B50E0001210F008E
:10A3D0008740114A0400D368FD43BB43D360831E0A
:10A3E0008B4201D8FFF7E0FF00212000FFF72EFF8E
:10A3F0000A4A0B4B5168012E05D139431B19516094
:10A400005E700020F8BD2940516002221C19627064
:10A410009A6915409D61F4E70038004000800040D3
:10A420007860FF1F012210B58240074B002906D03B
:10A4300019680A431A600121FFF7C6FF10BD1968A9
:10A4400091431960F7E7C046008000400C2370B5C7
:10A45000002543430A4A29009B181D70094B04003C
:10A460001B185D70FFF7B0FF0123A34006492800C9
:10A470000A681A430A6005490A689A430A6070BD6F
:10A480009460FF1F7860FF1F3480004030800040E0
:10A4900070B504000E00FF2813D003250540FFF718
:10A4A000D5FF084AA3089B009B183F22ED00AA4055
:10A4B000AE40196820009143314319600121FFF734
:10A4C0008DFE70BD18380040F8B50C244443134B82
:10A4D0000500E4186368002B03D1A3681220002B49
:10A4E0001AD0022201270E4B00215B195A70280056
:10A4F0002770FFF769FF63681E1E08D0A3683E003F
:10A50000002B04D02800FFF759FE4640F6B2280081
:10A510003100FFF709FE0020F8BDC0469460FF1F20
:10A520007860FF1FF7B5C420FF222B4B800019581D
:10A53000002491433F3A0A431A508022274F520287
:10A54000274E1A60274B1D5D002D21D0A31E012B25
:10A5500003D80121E0B2FFF727FF012D18D11F4BCF
:10A560009B69E3402B4213D0E3B218000193FFF73D
:10A5700025FE01000198FFF755FFE3B2143B022BC3
:10A580001DD801217156184A8D405369AB43536160
:10A590003B7F002B0DD0E5B22800FFF795FF280088
:10A5A000FFF70CFE7B7F0100834202D02800FFF7FB
:10A5B000A5FD01340C370236172CC3D1F7BD01219C
:10A5C00000237156F3568D40074A9B009B189A68EA
:10A5D000AA439A60DCE7C04600E100E07860FF1F14
:10A5E0003DBE00117960FF1F00F0004010B5012151
:10A5F0000400FFF7E9FE0123044A002011194B7003
:10A60000A34091690B43936110BDC0467860FF1F62
:10A6100070B50E0015000400FFF718FF0C2363430C
:10A62000094A20009B189D605E60FFF74DFFF021F6
:10A63000064B074A8900051E5A5002D02000FFF73A
:10A6400005FF280070BDC0469460FF1F0000FF1F7B
:10A6500059A1001170B5134D07202C78002C1FD183
:10A66000982221005200280001F0D6F80123C420CE
:10A67000FF222B700C4B80001C635C630B4B1C6037
:10A680005C600B4B195891433F3A0A431A508022A1
:10A6900052021A600D20074A074901F07DF9200097
:10A6A00070BDC0467860FF1F00800040A0F00040F1
:10A6B00000E100E025A5001125A3001170B51D00E3
:10A6C00002240C2910D8094ACA40D2070CD5FBF73E
:10A6D00045FF041E08D1059A04992800FBF75AFF8C
:10A6E000FCF7C8FDFFF728FB200070BD121000002A
:10A6F00030B50D7802232C009C43184201D02B4327
:10A700001C0008252300AB43284201D02B00234323
:10A7100020241D00A543204201D01C4325002A23EC
:10A720000D70184204D011781E3B0B43137030BDDE
:10A730000028FCD10C2113788B43F7E7F8B51D00F6
:10A7400006AB1B88140007AA0E000B201778002BFD
:10A7500027D10A78022A49D14A6850781178000234
:10A76000244A08438018042840D800F075FF0312DB
:10A770001D1B2300F06801F027F8021CC0B2B8428C
:10A7800000D93A1CD2B22000F1682A8001F0B4F955
:10A7900006E00222F3681B882A8023701B0A63707C
:10A7A0000020F8BD0622EEE701232B80F3681B781A
:10A7B0002370F5E7F368002B16D008222A801A8848
:10A7C00022701A88120A62705A88A2705A88120A75
:10A7D000E2709A8822719A88120A6271DA88A271EC
:10A7E000DB881B0AE371DBE72B80D9E701202B8094
:10A7F000D7E7C04600D6FFFFF7B516000A781D0060
:10A8000008AB1F880C000123022A18D14A6850782F
:10A81000117800022B4A0843801803280FD800F053
:10A820001BFF02254439E06800F0CEFFC0B20723C9
:10A83000B84204D37B190193152B02DD0D231800B8
:10A84000FEBDE0682A003100C01901F055F96B46E1
:10A8500000209B88E268D0541B4B1B68834203D0C6
:10A860001B68834200D098470023E8E70B23002FA2
:10A87000E5D1022DE2D1737832781B021343E268EE
:10A880001380114B1B68002BEED01B68002BEBD004
:10A890000120E8E70B23002FD1D1062DCED12A00CD
:10A8A0003100E06801F028F9DEE70B23002FC6D164
:10A8B000012DC3D132787533012AC0D8E3681A70EC
:10A8C000D2E7C04600D6FFFF8462FF1F70B50C00C0
:10A8D0001500072837D800F0BFFE041436361B36A3
:10A8E000242E182015290BD8184E162200213000CE
:10A8F00000F03AFF22002900300001F0FDF80020AE
:10A9000070BD18200229FBD11288114B1A80F6E77E
:10A9100018200829F4D10A000E48290000F08CFE06
:10A92000EDE718200129EBD10B4B10780B49DA69C0
:10A93000FFF7DEFEE3E718200129E1D1064B10788E
:10A940000749DA6BF4E70220DAE7C0466C62FF1FC2
:10A95000523EFF1F483EFF1FD83DFF1F003EFF1F16
:10A96000203EFF1F030010B50020DB0704D50721A0
:10A97000024A034800F08CF810BDC046C8BE001162
:10A98000D83DFF1F054A03001068002803D08288C5
:10A990009A4201D1806870470068F6E77C64FF1F27
:10A9A0000A88030008009A4204D08A8804309A4238
:10A9B00000D0002070470000F8B5F22200230D4FB0
:10A9C0000D4E7968050042433370994200D07B6098
:10A9D0000A4C0021200000F0C7FE00231A007C6012
:10A9E000AB4202D100203370F8BD01332280DBB2CC
:10A9F000F234F5E77465FF1F7265FF1F8064FF1F67
:10AA000073B56B4601900600684615001980FCF787
:10AA100063FF041E11D1002D0FD07689002E11D0B6
:10AA20000C2000F0C9FE00280ED0084A046013680C
:10AA300086808560002B02D11060200076BD1A0050
:10AA40001B68F7E70224F8E71324F6E77C64FF1F8E
:10AA5000012100220A4B10B549420A4C1980998005
:10AA60009A719A70084B2070012019805A60FFF784
:10AA7000A3FF2078FCF78EFF0448FDF749FF10BDC7
:10AA80008C62FF1F7C65FF1F7465FF1F3DAB0011CB
:10AA9000022310B5002802D0FFF7B2FF0300180010
:10AAA00010BD0000030010B50020DB0704D5042111
:10AAB000024A0348FFF7A4FF10BDC046DCBE0011E8
:10AAC000583EFF1FF0B50E2687B003930CAB1F88CE
:10AAD00002ABF6180500080031000292FDF77EF87F
:10AAE00004000120002C0FD03088FFF74BFF03003B
:10AAF0000E20002B08D05E68002E05D02100280013
:10AB0000039B029A0097B04707B0F0BD0A4B10B5FF
:10AB1000984207D10122002352420A808B708A801A
:10AB20008B7110BDFFF73CFF0028FAD001235B4278
:10AB3000038000238370F4E7FFFF0000F8B50500F1
:10AB400001290AD1134E00243388F227AB4219D0D1
:10AB500028001149FFF7DAFF06E0022904D1013984
:10AB6000FDF754FF0028EDD0F8BD3B006343726849
:10AB7000D018D35A002B09D03A00002100F0F4FD80
:10AB80000134E4B2054B1B78A342EED801235B42AB
:10AB90003380DDE77465FF1F8C62FF1F7265FF1F46
:10ABA00010B5FFF7FDFE03000020834200D0987827
:10ABB00010BD0000F0B589B01C000EAB80CB039037
:10ABC0001E8810AB1B78049202930B7A0D00DB06F3
:10ABD00016D42B780593022B24D00498FFF7D2FECD
:10ABE000002812D003689C46002B0ED0029B220046
:10ABF000019329003B00644603980096A04705E0B6
:10AC00000498FFF7BFFE002802D10E2009B0F0BD66
:10AC10008368002BF9D00A2229000398984700285E
:10AC2000D7D0F3E76B6858781A786B4B0002104363
:10AC30009842D2D8043B984210D2684B984242D0F6
:10AC400015D8674BC0180128C7D80B20002EDDD1BE
:10AC5000EB681A7859683A80200028E0614BC018E8
:10AC6000032800D979E000F0F7FC846A789E5E4BF7
:10AC70009842B2D10B20002EC8D101233B80EB6853
:10AC800031001B7823706889013080B2FCF7A6FF81
:10AC90003A88031E0ED0017802328A183A8042891F
:10ACA00062704289120AA27059680278E01C00F0B2
:10ACB00023FF06E004323A8031000422601C00F0D9
:10ACC00053FD0020A2E70B20002E9FD1EB6807A9BF
:10ACD0001E8804233B80330A300026706370FCF723
:10ACE0007DFF051E28D004AB9A890E2304A95B18AA
:10ACF0003E49C668FCF7E6FF00280BD12B783C489C
:10AD00006A680599FBF79CFB002803D1012304AA7C
:10AD10005B42D3813278022A06D17168201D00F08F
:10AD2000EBFE3B8802333B800E2304AA9B181B8852
:10AD3000A3701B0AE370C4E704ABDE81F4E70B20C9
:10AD4000002E00D062E7E9680398FFF729FF02238D
:10AD50003B802070000A6070B3E70B20002E00D00B
:10AD600054E70222EB681B883A8023701B0A637049
:10AD7000A7E7E86800F028FDC2B203000720B2424E
:10AD800000D243E70DD00299DBB27118994202DB81
:10AD9000921BD3B20293029BE9681A003B80891987
:10ADA0005AE70023F6E70B20002E00D02EE70722FB
:10ADB000EB683A801A7822705A7862705A88A270CA
:10ADC0005A88120AE2701A792271DA886271DB8875
:10ADD0001B0AA37175E7C046042900000228000081
:10ADE00000D8FFFFFFD6FFFF03280000FFFF000091
:10ADF0000CBE0011F0B58DB06B46002008912022EA
:10AE00009B5E83423DDAA64B187800F02DFE071EAC
:10AE100032D00378B02B2CD10079023816281FD8F5
:10AE200000F00AFD17001E001E001E0031001E006B
:10AE300096001E001D011E0052011E0073011E001F
:10AE4000CD011E0050021E001E001E008E021E00BC
:10AE5000E302944B94491B8878880B80FBF730F809
:10AE60003800FCF7B1FF914B1B68002B01D0380074
:10AE70009847380000F080FE8020089B0002434085
:10AE800018000DB0F0BDEE220021874800F06CFCE8
:10AE90000BAA3B7B7989388900923A000D32FCF786
:10AEA000B5FD0400804B1B78002C3FD146E0804B61
:10AEB000788805937F4B4100CB5A0BAE073BDBB242
:10AEC00032880293002301937B4B21000693009369
:10AED000059BFFF76FFE744D002810D1069B3A8A40
:10AEE0001B889A420BD138000599123000F0F4FB10
:10AEF000002804D02B7862899B00EB185A80162317
:10AF000006A81B18328820007989FCF7DBFE2B7815
:10AF100004009A00AA1851880029C3D00133DBB27B
:10AF20002B70002807D006A9C98A9180634A12882D
:10AF30009A42BCD802E0012149429180002B04D002
:10AF400059497888FAF7F0FF8AE73E890A2479E0C0
:10AF500000253E89574B06937B88069A5B009B5AD7
:10AF6000033B9D4202DB002DF0D05BE0162206A8D9
:10AF700012183B7B798900923A0030000D32FCF7C1
:10AF800045FD0590002858D04689017A7888FCF75D
:10AF900007FD041E44D1464B78880793069B410069
:10AFA000C95A454B0439C9B206AAD28A06930291FE
:10AFB000019400930599079BFFF7FCFD041E2FD118
:10AFC000069B39491A88931C002D26D14B8079881D
:10AFD000384B4900CB5A5119033B8B4220DD059B6E
:10AFE00031485B8941190B71A91C0135C9B2EDB219
:10AFF000059145191B0A2B71059B2D49043318181F
:10B0000000F07AFD2C4B059A1B88D318DDB22C4B2F
:10B010009E4205D00136B6B29CE749889942D6D007
:10B02000002D0CD0204C2800618800F0BDFA207063
:10B0300021007888FAF788FF12E7059CF0E7002CDA
:10B0400000D183E77B78142B00D109E716493B79BF
:10B050004E800B700C717888FAF728FF00E71624F1
:10B0600006ABE41821003889FCF7B8FD011E00D1B9
:10B07000B7E1788822880F4C45002C5B0A4D013CD3
:10B08000E4B2029400240F4B01940095FFF792FD67
:10B09000041E00D014E129007888FAF765FFDFE686
:10B0A0007C65FF1F483DFF1F9462FF1F8862FF1FE2
:10B0B0008863FF1FC45EFF1F7864FF1F463DFF1FAC
:10B0C000FFFF00009662FF1F162406ABE418210064
:10B0D0003889FCF783FD011E00D182E1788822883F
:10B0E000AE4C45002C5BAE4D013CE4B202947C8931
:10B0F000AC4B01940095FFF75DFD041E00D0DFE02E
:10B1000029007888FAF73AFFAAE60025A44B1D80AB
:10B110003B00F6331B78A24A78880792AB4208D9E5
:10B120009E4B12880693069943005B5A013B9A4254
:10B1300003DB0799FAF72CFF92E616246B00FB1845
:10B14000059306ABE418059B21001889FCF746FD22
:10B15000011E03D1059B01241E8973E77888924B59
:10B160002288069C099343001B5B904E013BDBB297
:10B170000293002300960193099BFFF71BFD041E19
:10B1800002D0059B1E895DE77B88069A5B009B5A6F
:10B19000079A108832881218934202DC1B1A013B6E
:10B1A00033807F4C023032880999001900F0A4FCEA
:10B1B0002388328801359B182380EDB2A8E70BAABB
:10B1C0003B7B7989388900923A000D32FCF71EFCEE
:10B1D00000250590059B002B04D10A24002D00D1E9
:10B1E0006EE060E0059B7888197AFCF7D9FB0100D6
:10B1F000041E63D1694C6C4B788806940993069BB6
:10B200004400E45A694B063CE4B20BAE3288079323
:10B210000294019100930599099BFFF7CBFC041E52
:10B220004CD1079B5E491B881A1D002D30D14A80E6
:10B23000059B5B4C5A8963191A716B1C9BB2E3180E
:10B24000120A1A71162306A832881B1879890598E4
:10B25000FCF738FDFF21AA1C2E1D03350B000590BD
:10B2600092B2B6B2ADB2002803D006ABDB8AD9B237
:10B270001B0AA218651911712B714C4D301D2A88BB
:10B280004949201800F038FC2B88F618B5B2A1E720
:10B290004988914207D17A8806995200525AEB1890
:10B2A000053A9A42C4DC3E4C2800618800F0ACFBB1
:10B2B000207021007888FAF775FED1E5002DF2D1D3
:10B2C0003E89BFE6162606ABF61831003889FCF732
:10B2D00085FC3D000400FA3500282DD0037A9B063A
:10B2E0000CD400227B893989788800923A000C328C
:10B2F000FFF7E8FB041E10D03E8915E03088FFF709
:10B3000041FB00281AD08368002B17D0210012229D
:10B3100078889847041EE4D0EEE72B78002B02D102
:10B320007888FAF74FFE00262B78002B00D097E59F
:10B33000002C00D194E585E60124DDE70E24DBE74F
:10B34000162506ABED1829003889FCF747FC041ECA
:10B3500047D0037A9B0611D4154A7B8811889942FD
:10B3600003D01448814207D11380134BF2261D7875
:10B370000023D9B2A94221D30924A1E72888FFF7E5
:10B3800001FB00282FD08368002B2CD02100122233
:10B3900078889847041EDFD092E7C046C45EFF1F3E
:10B3A0009462FF1F9662FF1F8863FF1F7864FF1F70
:10B3B0007465FF1FFFFF00007265FF1F31005943D6
:10B3C000546801336018615A0029D2D13C00083416
:10B3D0002100F22200F090FB21007888FAF7FAFDB4
:10B3E0003EE501246CE70E246AE71D4B1A887B8832
:10B3F0009A4231D07888FAF7F7FD31E5F2230598C3
:10B4000051684343CD18C95A00291FD03B7A012BFC
:10B410000BD16C88AB887888AA1D0094FFF752FB8B
:10B42000041E02D000233B722E88F2220021280045
:10B4300000F09AF900232B80059B0133DBB20593C2
:10B44000084B05991B78064A8B42D7D801235B42EB
:10B450001380002CCED0F5E5002634000596EFE7EA
:10B460007465FF1F7265FF1F70B504000E001500A4
:10B47000FFF796FA031E08D131000548FFF790FA4E
:10B4800003001120002B02D01C8000209D7070BD95
:10B49000FFFF0000F8B50B4F06003B780D001400CD
:10B4A000FF2B0ED00A2000F02FF9011E09D0B12386
:10B4B0000380002346800371C5800481387800F042
:10B4C00013F9F8BD993EFF1FF7B50F0008A9060054
:10B4D000088809A90B240988002821D10234022BED
:10B4E0001ED1557813782D021D432B008B430193F9
:10B4F0007334002B14D1FB68300019000093FFF760
:10B500004FFB019C85420BD02A0030000099FFF7C9
:10B51000ABFF041E04D12A0030007989FFF7BAFF7F
:10B520002000FEBDF0B50E7885B003900AA805880E
:10B530000120022E0DD14C682778647824023C4308
:10B54000054FBC4205D10398DBB201960095FFF789
:10B55000BBFF05B0F0BDC04602290000034B10B58B
:10B560001B68002B00D09847FEE7C0468065FF1F90
:10B5700007B501A8FFF7F2FF044A05480021121A97
:10B5800000F04AF9F8F736F9FEE7C0468465FF1F78
:10B590009C3EFF1F0000000001B40248844601BC2D
:10B5A000604700BF8B52010001B40248844601BCD1
:10B5B000604700BF350E000001B40248844601BC5C
:10B5C000604700BFC51D000001B40248844601BCAD
:10B5D000604700BF291C000001B40248844601BC3A
:10B5E000604700BF2526000001B40248844601BC24
:10B5F000604700BF392BFF1F01B40248844601BCDD
:10B60000604700BF055E000001B40248844601BCEB
:10B61000604700BFEDA5000001B40248844601BCAC
:10B62000604700BFE117000001B40248844601BC36
:10B63000604700BFC521000001B40248844601BC38
:10B64000604700BF810E000001B40248844601BC7F
:10B65000604700BF350E000001B40248844601BCBB
:10B66000604700BF4D36FF1F01B40248844601BC4D
:10B67000604700BFD91B000001B40248844601BCEA
:10B68000604700BF9DA9000001B40248844601BC88
:10B69000604700BF6DBC000001B40248844601BC95
:10B6A000604700BF017F000001B40248844601BC2E
:10B6B000604700BF5118FF1F01B40248844601BC17
:10B6C000604700BFADAE000001B40248844601BC33
:10B6D000604700BFDD66010001B40248844601BC3A
:10B6E000604700BFCD4C010001B40248844601BC54
:10B6F000604700BF594F010001B40248844601BCB5
:10B70000604700BF8552010001B40248844601BC75
:10B71000604700BF1D4D010001B40248844601BCD2
:10B72000604700BF0124000001B40248844601BC08
:10B73000604700BFB54C010001B40248844601BC1B
:10B74000604700BF5522000001B40248844601BC96
:10B75000604700BF311B000001B40248844601BCB1
:10B76000604700BFE12AFF1F01B40248844601BCC4
:10B77000604700BF154D010001B40248844601BC7A
:10B78000604700BFA54F010001B40248844601BCD8
:10B79000604700BF1147010001B40248844601BC64
:10B7A000604700BF090E000001B40248844601BC96
:10B7B000604700BF4D1F000001B40248844601BC31
:10B7C000604700BF3D4B010001B40248844601BC04
:10B7D000604700BFDD52010001B40248844601BC4D
:10B7E000604700BF3936FF1F01B40248844601BCE0
:10B7F000604700BF5933FF1F01B40248844601BCB3
:10B80000604700BF1D4B010001B40248844601BCE3
:10B81000604700BFB130FF1F01B40248844601BC3D
:10B82000604700BFB70E000001B40248844601BC67
:10B83000604700BF8D12000001B40248844601BC7D
:10B84000604700BF6136FF1F01B40248844601BC57
:10B85000604700BFE548000001B40248844601BCCF
:10B86000604700BF4550000001B40248844601BC57
:10B87000604700BF456B010001B40248844601BC2B
:10B88000604700BF75A9000001B40248844601BCAE
:10B89000604700BF7D18FF1F01B40248844601BC09
:10B8A000604700BF5125000001B40248844601BC36
:10B8B000604700BF014C010001B40248844601BC4E
:10B8C000604700BF3555000001B40248844601BC02
:10B8D000604700BFE528FF1F01B40248844601BC51
:10B8E000604700BF4551010001B40248844601BCD5
:10B8F000604700BF212DFF1F01B40248844601BCF0
:10B90000604700BF492DFF1F01B40248844601BCB7
:10B91000604700BFC56D010001B40248844601BC08
:10B92000604700BF9134FF1F01B40248844601BC48
:10B93000604700BFD949010001B40248844601BCF8
:10B94000604700BF156B010001B40248844601BC8A
:10B95000604700BF5549010001B40248844601BC5C
:10B96000604700BF2951010001B40248844601BC70
:10B97000604700BFC9A9000001B40248844601BC69
:10B98000604700BFB14E000001B40248844601BCCC
:10B99000604700BFB131FF1F01B40248844601BCBB
:10B9A000604700BF812BFF1F01B40248844601BCE1
:10B9B000604700BFA946010001B40248844601BCAB
:10B9C000604700BF5147010001B40248844601BCF2
:10B9D000604700BF2146010001B40248844601BC13
:10B9E000604700BF851F000001B40248844601BCC7
:10B9F000604700BFC94A010001B40248844601BC47
:10BA0000604700BF6D33FF1F01B40248844601BC8C
:10BA1000604700BF090E000001B40248844601BC23
:10BA2000604700BFC926000001B40248844601BC3B
:10BA3000604700BF0D35FF1F01B40248844601BCBA
:10BA4000604700BF7918000001B40248844601BC79
:10BA5000604700BF5D17000001B40248844601BC86
:10BA6000604700BFBD30FF1F01B40248844601BCDF
:10BA7000604700BFF54E010001B40248844601BC96
:10BA8000604700BFF92AFF1F01B40248844601BC89
:10BA9000604700BFF30E000001B40248844601BCB9
:10BAA000604700BFF94C010001B40248844601BC64
:10BAB000604700BF5952010001B40248844601BCEE
:10BAC000604700BF2534FF1F01B40248844601BC13
:10BAD000604700BFE130FF1F01B40248844601BC4B
:10BAE000604700BF691F000001B40248844601BCE2
:10BAF000604700BF3935FF1F01B40248844601BCCE
:10BB0000604700BFE94C010001B40248844601BC13
:10BB1000604700BFED4A010001B40248844601BC01
:10BB2000604700BF0D52010001B40248844601BCC9
:10BB3000604700BF6532FF1F01B40248844601BC64
:10BB4000604700BFE533FF1F01B40248844601BCD3
:10BB5000604700BFA533FF1F01B40248844601BC03
:10BB6000604700BF2124000001B40248844601BCA4
:10BB7000604700BFB352010001B40248844601BCD3
:10BB8000604700BF434D010001B40248844601BC38
:10BB9000604700BF792EFF1F01B40248844601BCF4
:10BBA000604700BFE928000001B40248844601BC98
:10BBB000604700BF6571010001B40248844601BCC2
:10BBC000604700BF091B000001B40248844601BC65
:10BBD000604700BF056A000001B40248844601BC0A
:08BBE000604700BF3D180000A2
:10BBE800000101030202030304030502060207021F
:10BBF800080209030A030B030C020D000E030F03CE
:10BC0800100311031303140315001600B93B0011A8
:10BC1800ED3B001100000000020000002ABC0011EA
:10BC2800192A0F180A000000F1590000FD2400002D
:10BC380041460100198000112DA0001181740011E6
:10BC48001D7E001105530011F5AD00116D4F001157
:10BC5800AD3D0011DD3E0011000000001616000089
:10BC68000200000074BC0011F4FFF3FFD2FC0000D6
:10BC78001D400011000000000000000054757961AB
:10BC88000042312E340030303135006769746875F0
:10BC9800622E636F6D2F70767678005448303500C9
:10BCA80002000000BCBC0011292A282A272A262ABB
:10BCB800252A242A0A180000E20400007102000064
:10BCC80078EC0000744000001027000060F00000CD
:10BCD80006640000204E000000000000050000007F
:10BCE8001F501D00023CB4000001150014000000A4
:10BCF800A102000030313233343536373839414209
:10BD08004344454600000000095700115D570011E3
:10BD1800000000000200000028BD00116F2A6E2AF2
:10BD28001A18EAD8BC80F0FC60000000000000008F
:10BD38000000F303B59747D6F613F7D777E6F0A7D1
:10BD4800F474000001A00000000000006410B71D9A
:10BD5800C8206E3BAC30D9269041DC76F4516B6B31
:10BD68005861B24D3C7105502083B8ED44930FF0F3
:10BD7800E8A3D6D68CB361CBB0C2649BD4D2D386A9
:10BD880078E20AA01CF2BDBDFB349B5F80000080F6
:10BD98000010000000000000836000110D77001102
:10BDA800A7600011157B00112B610011EB7A0011BF
:10BDB800A1610011C17A0011F3610011897C0011A1
:10BDC8005B620011897C00118D620011437C0011B7
:10BDD800A1610011797A001119620011217C00110A
:10BDE8000000000000000000FF620011217C00112B
:10BDF8006163001125770011052A042A012A002A07
:10BE08000229032801280028011800180000000052
:10BE1800000000000000000000000087010102018E
:10BE280002010102010203030401030101010101EE
:10BE38000303020103000D000E001000110013009F
:10BE48001401070108010A010B011C011D0204026B
:10BE580005020702080219021A021C021D03010347
:10BE6800020317000201000504000807000B0A007E
:10BE78001716001D1C010201010504010E0D011118
:10BE880010011413011716011A19020201020B0AF4
:10BE9800020E0D02111002141302171603050403F3
:10BEA8000807030B0A030E0D0001020307090A0B1A
:10BEB8000E0F101112141718191A1B1F2021220017
:10BEC8003DA70011F9A700110000000002000000C2
:10BED80012BE00110000000025B50011000000008E
:08BEE8000200000010BE001171
:020000041FFFDC
:1000000000000000153D001130BC00112CBC001197
:10001000A85BFF1F000000000000000000000000BF
:1000200000000000000000000000000000000000D0
:1000300000000000000000000000000000000000C0
:1000400000000000000000000000000000000000B0
:1000500000000000000000000000000000000000A0
:100060000000000000000000000000000000000090
:100070000000000000000000000000000000000080
:100080000000000000000000000000000000000070
:100090000000000000000000000000000000000060
:1000A0000000000000000000000000000000000050
:1000B0000000000000000000000000000000000040
:1000C0000000000000000000000000000000000030
:1000D0000000000000000000000000000000000020
:1000E0000000000000000000000000000000000010
:1000F0000000000000000000000000000000000000
:1001000000000000000000000000000000000000EF
:1001100000000000000000000000000000000000DF
:1001200000000000000000000000000000000000CF
:1001300000000000000000000000000000000000BF
:1001400000000000000000000000000000000000AF
:10015000000000000000000000000000000000009F
:10016000000000000000000000000000000000008F
:10017000000000000000000000000000000000007F
:10018000000000000000000000000000000000006F
:100190006D2DFF1FCD2BFF1FC16601000000000069
:1001A000000000000000000000000000000000004F
:1001B000000000000000000000000000000000003F
:1001C000000000000000000000000000000000002F
:1001D000000000000000000000000000000000001F
:1001E000000000000000000000000000000000000F
:1001F00000000000000000000000000000000000FF
:1002000000000000000000000000000000000000EE
:1002100000000000000000000000000000000000DE
:1002200000000000000000000000000000000000CE
:1002300000000000000000000000000000000000BE
:1002400000000000000000000000000000000000AE
:10025000000000000000000000000000000000009E
:10026000000000000000000000000000000000008E
:10027000000000000000000000000000000000007E
:10028000000000000000000000000000000000006E
:10029000000000000000000000000000000000005E
:1002A000000000000000000000000000000000004E
:1002B000000000000000000000000000000000003E
:1002C000000000000000000000000000000000002E
:1002D000000000000000000000000000000000001E
:1002E000000000000000000000000000000000000E
:1002F00000000000000000000000000000000000FE
:1003000000000000000000000000000000000000ED
:1003100000000000000000000000000000000000DD
:1003200000000000000000000000000000000000CD
:1003300000000000000000000000000000000000BD
:1003400000000000000000000000000000000000AD
:10035000000000000000000000000000000000009D
:10036000000000000000000000000000000000008D
:1003700071B5001100000000000000000000000046
:10038000000000000000000000000000000000006D
:10039000000000000000000000000000000000005D
:1003A000000000000000000000000000591AFF1FBC
:1003B000000000000000000000000000000000003D
:1003C000000000000000000000000000000000002D
:1003D000000000000000000000000000000000001D
:1003E000000000000000000000000000000000000D
:1003F00000000000000000000000000000000000FD
:081838009069FF1F4118FF1F1A
:10184000024981F3088802F097F800009069FF1FB1
:1018500010B502F069F8072804D0122808D0022831
:1018600008D010BD044A0420136B01331363F8E75A
:101870000220F6E71420F4E76C5FFF1FF8B50700BD
:101880000C0026002500503630785135002804D150
:101890000300287058342370F8BD2978CA00481E08
:1018A0008141A3183800A25C5B68C9B2FFF7D0FF82
:1018B00000280DD12B78DA00A218013350602B706C
:1018C0003378044A013B3370136A01331362D8E75B
:1018D0000123DFE76C5FFF1F5C234343074910B51B
:1018E000C9180B0058331B78012B05D1FFF7C6FF31
:1018F000034A936A0133936210BDC046A05FFF1F85
:101900006C5FFF1F10B501F0EFFF064A01211300C5
:1019100010CB4942D967044B136002F08DF82000C8
:1019200010BDC04600E100E01000100010B504003A
:1019300001F0DAFF024B1C6002F07EF810BDC046D9
:1019400000E100E0431E5A425341A022F0B5D2010B
:101950005B421340154D164A40019B182A18127E0F
:101960008BB00191002A1BD01A000832D46F0022DC
:10197000E6B206AFE4B294420EDC2818C369002B2D
:1019800008D0019902AA117106AA049202AA16733C
:1019900003A898470BB0F0BD1978B9540132EAE7B3
:1019A0001A7D1A7806AB01261A70E6E72C62FF1F33
:1019B00000400040F0B5254B04004001C25C85B0FA
:1019C000002A2BD01A18117E002927D0917E0029D9
:1019D00024D01179022921D11689D788D168F51B25
:1019E000ADB22A1C102D00D9102292B2BE4217D1DE
:1019F0001818012303710023C269C38003819A422E
:101A000006D06846032103730171029301A8904731
:101A10000820002C00D0192001F08EF805B0F0BD90
:101A2000013C65426C41A0256442ED012C40084D0B
:101A30001B186419074D0633013A92B2AA42EDD041
:101A40001888461C1E80085C2070F5E72C62FF1F7A
:101A500000400040FFFF00000F220E4B10B59868B9
:101A6000104002380A280BD801F0F0FD0D0A0B0ACD
:101A70000A110A0A0A0A060002210020FFF762FF83
:101A800010BD0121F9E70020FFF794FFF8E7DB6FB5
:101A9000F6E7C046004000400F220E4B10B5986894
:101AA000104002380A280BD801F0D0FD0E0A0B0AAC
:101AB0000A120A0A0A0A060002210120FFF742FF61
:101AC00010BD01210800F9E70120FFF773FFF7E7D8
:101AD000DB6FF5E700900040564B70B51B68012B9B
:101AE00003D1554A936D0133936501F0F5FE534BD5
:101AF000534A1860534B544C1A600123534A1360E5
:101B0000534A13602378002B06D0062251495248CD
:101B100001F0B2FE00232370504A514B10681B782D
:101B2000C1B2002B0ED14F4CC0B223785BB2002B58
:101B30004FDB237824785BB264B21B0424021B19A8
:101B40001B1813600B1C50294ED95023464A474995
:101B50001078DBB2FF2202284BD10868444C454D77
:101B6000267890432A78964254D9227824782E7881
:101B7000023B5D10A31B6B435201D31A10335B1160
:101B80001843086001F078FD031F012B45D83A4B3C
:101B90001B78002B06D0394B1B78002B02D000207D
:101BA00001F022FEA122364B92009978354B4A4330
:101BB0001B689B18832292009B181B78033B012B08
:101BC00003D8AF20400001F0E7FD01222E4BDA825E
:101BD00070BD237824785BB264B2FF33FF341B04FA
:101BE00024021B190138ABE7CAB2022AAED2022383
:101BF000ACE70868254C264D267890432A78964213
:101C000008D9227824782D78023B5B10641B63434B
:101C10005201B2E72378DBB2B2E70228D5D11D4BDF
:101C20001B78013B022B03D91B4B1B78022BCCD119
:101C30006C20C8E79809FF1FFC0FFF1FA45EFF1F61
:101C4000FF3F000014100340A85EFF1F0C1003406C
:101C500000100340D50BFF1F7211FF1FB40003409B
:101C60008C09FF1F680AFF1F490AFF1F94000340E9
:101C7000460AFF1F470AFF1FF908FF1F2209FF1F1F
:101C8000300DFF1F3409FF1FBC0BFF1F440AFF1F4D
:101C9000450AFF1F1C09FF1F2309FF1F10B501F094
:101CA000FBFD0022014B1A8010BDC046A05EFF1F45
:101CB00070B5244D2B68002B28D001F075FE2B68E1
:101CC000D8402B680400002B27D001F09DFE2B6824
:101CD000D8401D4B1D4A9978A1239B004B431268A5
:101CE000D118D25C91239B00002A20D0CA5801321F
:101CF000CA50174B17491B680868834214D3D23B5C
:101D0000181A012A1AD0144B186070BD01F04CFE4D
:101D1000124B196801F050FED3E701F075FE0F4B2E
:101D2000196801F049FED4E70D495B18E8E7CA508D
:101D30000C4B1B68DB68E418201AE4E7F530FF3031
:101D4000E1E7C0461C08FF1F300DFF1F3409FF1FCD
:101D50009C09FF1FA45EFF1FA009FF1F1808FF1F9B
:101D60002DFF3F00AC5EFF1F70B504000D00282959
:101D700016D10300A433C2881B889B1A0B4A9BB25E
:101D800093420DD906006A3605223100653001F014
:101D9000ABFC002804D13100200001F045FE70BDED
:101DA0002900200001F010FDF9E7C046FE7F000089
:101DB000F8B50500012001F007FE134CA36AA26AE2
:101DC0009342FBD1114E336001F066FC10490300D1
:101DD00008601048426894460F4A17680022BC45C4
:101DE00001D24268BA1A0D4802603268AD18A422C6
:101DF000E562606A520302436262094A1278002A6D
:101E000001D00F3B0B60F8BD00F00040340AFF1F0B
:101E1000E408FF1F28100040180AFF1F1C0AFF1FBC
:101E20001C09FF1F70B580241025E405A3682B430F
:101E3000A36001F0A9FDA368AB43A36070BD0000DF
:101E4000F7B5160080221C001023D205019191687D
:101E500005000B43936000225A4BD7301A6001F003
:101E6000D3FC9D232A002F009B00EB58CA3201218E
:101E70000092FC37002B01D00021009A386801F055
:101E80003BFD2900009BCB311A784F4BD3351A60AC
:101E90004B780A781B0213438A7812041A43CB78D2
:101EA0001B061343494A1BBA13604B790A791B027C
:101EB00013438A7912041A43CB7931001B0613436A
:101EC000434A1BBA13606B782A781B021343AA7823
:101ED00012041A43EB781B0613433E4A1BBA1360E5
:101EE000019A330213433C4A13603C4B22001B1BF4
:101EF0009C4603293DDCB3089A0013005142B21AF4
:101F0000032A46D1354AE018511A827840781204E3
:101F100000020243E05C043302430A600022FF2B0C
:101F20004BDDF0222E4B12011A600F222D4B1A604E
:101F30002D4A1368002BFCD00023224A2749136046
:101F4000091B321D0B191B68043A180A23706070B4
:101F5000180C1B0EA070E3700434002AF2DC8022FF
:101F600010213B68D20501333B6093688B4393603B
:101F7000F7BD6346D578981893782D061B042B433C
:101F8000157804392B43557804322D022B43036016
:101F9000AFE7022A0AD1114AE05C511AE2185278DE
:101FA000120202430A6004339BB2B7E7012AB5D19B
:101FB0000A4A521AE15C1160F5E7084959180A60AB
:101FC0000433ACE7000004403C0004403800044007
:101FD00034000440300004400C0004400001044080
:101FE000040004401000044014000440F7B515003C
:101FF00080221C001023D2050091916807000B433A
:1020000093600023654AD730136001F0FDFB9D23E8
:102010003E009B00F9583B00CA363200FC330029D1
:1020200000D07FE0586801F067FC390032785C4BE3
:10203000CB311A604B780A781B0213438A78AC467E
:1020400012041A43CB78281D1B061343554A1BBAAA
:1020500013604B790A791B0213438A7912041A43DD
:10206000CB791B061343504A1BBA13604B7A0A7A8A
:102070001B0213438A7A12041A43CB7A21001B06EF
:1020800013434A4A1BBA1360009A2B021343484A6F
:1020900013602200474B1B1B0093009BCE785B18FC
:1020A00001938B7836061B0433430E780438334390
:1020B0004E78043136023343019E33600328ECDC52
:1020C0000321A808431C9B002940800003292BD131
:1020D0003849E5185E18A9786D78E35C09042D028B
:1020E000294319433160030008330021FF2B2DDD04
:1020F000314B324919600F21314B196001232749B7
:102100000B60304B19680029FCD006211B680B407E
:10211000042B20D080220020D20593680A318B4303
:102120009360FEBD01217DE7022908D121495D1898
:10213000E1184978E35C090219432960D3E70129D2
:10214000D3D11C495918E35C0B60CCE71948181827
:1021500001600433CAE7002310490B606346002B7B
:102160000CDC3B00FC335A68102101325A6080229B
:10217000D205936801208B439360D2E7009B9B18A4
:102180001B68190A13705170190C1B0ED3700423AD
:102190005B4291709C440432E0E7C046000004407A
:1021A0003C00044038000440340004403000044047
:1021B0000C0004400001044004000440080F00002B
:1021C000100004401400044010B5002901D001F0B3
:1021D0004BFC10BDF7B5604B01919978A1239B0092
:1021E0004B435E4A060014681022E418D6235B00B5
:1021F000E0583623FF33E35C00279343222B41D181
:10220000574B0F3A1A600760012501F025FC019B2E
:102210001880E8235B00E35C002B01D0B34258DD5B
:102220000023504FFB70AD33FF33E3581A68002A88
:1022300003D09B88DB439B071DD03823FF33E35C2F
:10224000002B18D09B235B00E35C002B13D1D13310
:10225000FF33E35CB3420EDAA4235B00E15AE018DB
:10226000090A023101F070FB23000122FE33013E16
:1022700001351A87FA70E8235B00E35C002B2AD053
:10228000A8B2FEBD03683D00002BBED0818804309B
:10229000090A023101F058FBD6235B00E3581F60A6
:1022A000B2E72300B133BA00FF3398580137818871
:1022B0000430090A023101F047FBE8235B00E35CCC
:1022C000BB42EEDCE822F61AED1800235200A354BC
:1022D000A6E70027F1E7200001F02EFA00281FD022
:1022E000002E1DDD7319882647190193B6002000C2
:1022F00001F0DAFB5A3080002018406801358188EF
:102300000430090A023101F01FFB200001F0D4F96A
:10231000A3590133A351BD4202D0019B9D42E6D196
:10232000114BE35C002BABD095239B00E35C002BAF
:10233000A6D00E4BE15A0029A2D00D4AA35C9942C7
:1023400002D90133A3549BE700231A212000A35490
:1023500001F0BAF994E7C046300DFF1F3409FF1FA2
:1023600000140340E010FF1F5A0200007202000038
:102370005E0200000D4970B54A6E0D4CD2038B69A8
:10238000D20BA24206D80B4D0224AA4204D901F076
:102390005BFA70BD02246442E21815007E242540D9
:1023A0002242F4D0A3432B438B61F0E700F00040BE
:1023B0000A200000FC1C00000B001B3B70B5040051
:1023C0003020E02B0DD81300E025493BFF3B9BB2AA
:1023D000ED00AB4205D8034B200019825A8201F070
:1023E0008BF970BD8410FF1FD722044B92009B58BD
:1023F00010B5002B00D0984710BDC0460000FF1F4D
:1024000010B501F0ADF8FFF7EFFF2749274BCA6D74
:10241000274C1A4084235B001343CB65254B1B6874
:10242000186A01F0D1FA244B244A1A60244B254A39
:102430001A60A022244B52001A60244B187801F035
:10244000DBFA2000224901F0AFF90023A360023338
:10245000A360204B2049236003232048A36001F0A0
:10246000A3F910221E4BFF201A60802252031A602B
:10247000802292031A60802212041A6001F0B4F9DB
:10248000012001F0C9F9FA20400001F065F9582057
:1024900001F082F9134801F03FF9012001F0C4F97D
:1024A000072001F0F1F910BD00F0004000FEFEFF32
:1024B00014100040AC5EFF1F000003400180063D89
:1024C000BC00034034080000A40003404A0AFF1F78
:1024D00071020000C3090000FFFF3F002810004008
:1024E00000E100E030750000674E336888331B68F8
:1024F00083F3088801F0B8F9644A6549136800203D
:102500000B401360634B644A1B68934200D1A6E002
:1025100001F0BAFA0221614A13688B431360FFF796
:102520006FFF5F4B5F4C1878C0B201F00DF90023CC
:10253000A3600233A3605C4B0120236001F044FAE6
:102540000323A36001F020F9040001F0C5F90500A0
:1025500001F01AF9554B186001F01EFA544B196836
:10256000621A531EA14200D213008022D20393426A
:1025700001D39B029B0A3268D16AC90700D471E07B
:102580004C491C0C09689BB24C4359432402090A6C
:10259000641803264849FC3293680A6847489B1A26
:1025A000474A0768126847499B18474A9A183340B8
:1025B0009208DB190A600360042B03D9013233400F
:1025C0000A6003600E684149A619300001F0F4F971
:1025D0003F4F3E493B68C3183B603000019301F018
:1025E00093F93C4E3068081838493060884205D964
:1025F000019B01333B6001F087F9316001F0ECF998
:10260000354B1B78002B0DD001F066F9334B621B64
:10261000196812188A4232D24919091B091A30481E
:1026200001F0C2F82F4E337A002B0ED001F054F98E
:10263000621BF1681218914224D94919091B091A21
:10264000294801F0B1F800233372284B83F308883E
:1026500001F02AF8002001F017FA01F0BDF801F0AE
:1026600013FA5CE7DC0199000234641A5900641A19
:1026700009214B438033CB40A408E41889E7FA21B1
:102680008900CCE71A49DBE7AC5EFF1F1CF0004075
:10269000FFFFC1FF0C0AFF1FB641210310000040DD
:1026A000490AFF1F14100040C3090000100AFF1F51
:1026B000340AFF1F380AFF1F200AFF1F280AFF1FC6
:1026C0001C0AFF1F240AFF1FC4090000710200003A
:1026D0006008FF1F2C0AFF1F1C09FF1FE408FF1FD3
:1026E00000100040740BFF1F3C1000400000002051
:1026F000DC050000A022054B92009B5810B5002B72
:1027000001D0984710BD00F0E7FFFBE70000FF1F76
:10271000A122054B92009B5810B5002B01D0984781
:1027200010BD00F0D9FFFBE70000FF1FA222054B00
:1027300092009B5810B5002B01D0984710BD00F0B7
:10274000CBFFFBE70000FF1FA322054B92009B5825
:1027500010B5002B01D0984710BD00F0BDFFFBE77E
:102760000000FF1FA422054B92009B5810B5002BC0
:1027700001D0984710BD00F0AFFFFBE70000FF1F3E
:1027800070B501F0A9F84F4B186001F05DF9040035
:10279000C30702D401F060F870BD00224A4B1A60F2
:1027A0004A4B18780138042829D800F04FFF03203D
:1027B000181C2400200001F05FF90128ECD0444CE3
:1027C0002378042B6ED101F027F90028E4D000F023
:1027D0009BFF582000F0E0FF02232370DCE720007D
:1027E00001F0C2F8E9E7200001F006F8E5E7200073
:1027F00001F022F8E1E7200001F05EF9DDE700F0EA
:102800003BFF0500012808D1324B1B78053B012B0B
:1028100003D82000FFF76EFFD1E72D4B1B78022B6A
:1028200001D0052B20D1022D28D12B4B9B7BAB4314
:102830001CD12000FFF76CFF264B18780128BED171
:102840006405BCD4244925224B7B034205D1233A9D
:1028500013405A42534126331A000B7D9342AED99E
:10286000322001F031F8AAE7022D07D1194B1B786D
:10287000052B11D12000FFF759FFDDE7012D0BD10A
:10288000012B03D12000FFF75FFF98E7062B03D150
:102890002000FFF767FF92E7200000F01DFF022DE8
:1028A0008DD1C9E7032B04D10C4B987C01F034F88F
:1028B00072E7072B00D06FE7094B987B00F034FFDD
:1028C0006AE7C0469C09FF1F9809FF1F9009FF1F78
:1028D0002309FF1F1C09FF1FA60BFF1FBC0BFF1FB7
:1028E000D40BFF1F10B500F099FE10BDF7B50B0C0F
:1028F000FF270122009300233C001E001D00944688
:10290000019089B262469A4010000840184136187A
:10291000B6B2FF2F02D1012E00D19FB20098024023
:102920001A41AD18ADB2FF2C02D1012D00D19CB2DD
:102930000133102BE6D10320012E07D1012D04D144
:10294000019B2401E4191C700138FEBD102EFCD13E
:102950000238102DF9D00230F7E700008023F7B5D8
:102960009C46264B264F01932649274A274D284C43
:10297000284B02281AD1604638600868264E30403D
:10298000802636033043086001990978002909D16F
:102990001660224A2A60224A2260E0221968914386
:1029A000A03A1BE08021C9021160F2E766463E6052
:1029B0000F68194E3E408027FF023E430E6001998A
:1029C000097800290DD1176001280ED1154A2A6017
:1029D000154A2260E02219689143C03A0A431A60FE
:1029E000F7BD802189021160EEE7E0210F4A024322
:1029F0002A600F4A22601A688A43F0E74B0AFF1FD9
:102A0000E0000340D8000340900003400000034072
:102A10005000034040000340FFFFE3FF0280063DFB
:102A2000804508220180063D8066082200800698C5
:102A300080550822F8B51E4B80261A680020140025
:102A40003440324232D11A681A4F32431A6001229E
:102A50003B68063093433B6000F0B6FF0122164D01
:102A60002B681E432E603B680A2613433B60802779
:102A7000BF00124B1B683B4211D1013EF6B2FF2E44
:102A800009D17E220E4B1C682B68E40B1440934343
:102A900023432B6005E0082000F096FFE9E7002EB5
:102AA000EFD180222B68600893432B60F8BDC046AD
:102AB000C4F000405CF0004018F0004068F00040B6
:102AC00060F0004010B500F0EFFE01215820034AED
:102AD00000F0E2FFFFF7AEFF10BDC046600AFF1F27
:102AE00010B578220021034800F0E6FE00F034FF24
:102AF000002010BDB461FF1F70B5040000F0F4FEAB
:102B000000230C200B4A010059438D18515C002909
:102B10000DD0A14208D1012300246B7000F064FFA6
:102B200000F08AFF200070BD01330A2BEBD1122484
:102B3000F6E7C046B461FF1F70B5040000F0D4FE94
:102B4000002319001D000D4A1078002806D0A0426D
:102B50000CD1557001310C320A29F5D1002B0AD164
:102B600000F0FAFE00F068FF002070BD5078461EAD
:102B7000B0411B18EEE700F037FFF3E7B461FF1F29
:102B8000F7B504000C20002384460E4D01926746E1
:102B90005F43E85D7E19A04212D000280BD10A4B9A
:102BA0009C4662461B7808331370019B70707C55FD
:102BB0007160B360FEBD01330A2BE8D10320F9E751
:102BC0000720F7E7B461FF1FB061FF1F8020F8B551
:102BD000484BC0051B68C1248360474BFF251A681A
:102BE000012313434361454BA4001A68444B402121
:102BF0001A60444B1A68444B1A60444B1A59AA4352
:102C00001A51C52292009E58AE43314380269950F6
:102C10009F583F49F6010F403E439E509E588027E3
:102C20003602360A3043985080201A5900020A4072
:102C300002431A5104341A59364E3F04324080265A
:102C40003A431A511A5936061202120A32431A51DD
:102C500008341A5980260A4002431A51C3229200AE
:102C60009F58B446AF4337439F509F58294E0F405B
:102C700007439F509F5837408026360437438026AD
:102C80009F509F5836063F023F0A37439F50C0224D
:102C90001F59AF433A431A511A591202120A1643E6
:102CA000C6221E5192009C58AC4365462C439C5052
:102CB0009C5800250C4020439850C72080001A588B
:102CC000154C1140C02212020A431A50134B1B78B4
:102CD000DB08AB4201DC0020F8BD2378002B06D0D6
:102CE000A368002B00D0984701350C34EEE7122082
:102CF000F2E7C046D43DFF1FD03DFF1FB0F00040BB
:102D0000AC61FF1FB4F00040A861FF1F00E100E0CC
:102D1000FF00FFFFFFFF00FFB461FF1FB061FF1F57
:102D2000030010B51F2809D80722002013400724EC
:102D300004490A78A24313430B7010BD00230620F8
:102D4000F5E7C046B061FF1F054B06491B780A68CE
:102D500005485B0702401B0B134300200B607047C4
:102D6000B061FF1F1CF00040FFFFC1FF70B50C25D4
:102D7000FFF7EAFF0A4B1C780A4BE4086543ED189D
:102D8000002C01D1200070BD2B78002B06D06B6881
:102D9000002B00D09847013C0C3DF1E71220F2E7F0
:102DA000B061FF1FA861FF1F1FB5002102220B00A9
:102DB00001910091052000F0BFFD02230B490A6834
:102DC0001A42FCD120230393039B5A1E0392002B2B
:102DD000FAD1074A1368002BFCDA0B246C4420005C
:102DE000012100F071FE207804B010BD90C80040B1
:102DF00000C8004013B504000A4B0193019B002B4F
:102E000001D1112016BDFFF7CFFF2300034004427C
:102E100005D0052000F0D8FD019B013BEDE718002F
:102E2000F0E7C046FFFFFF0707B500F05DFD802219
:102E30000821D205936A0191002B01D107399162D3
:102E400002210C4A11600199481E01900029FAD113
:102E500003311160053101910199481E019000294B
:102E6000FAD11160002B02D18022D205936200F0CA
:102E7000E3FD07BD00C00040F0B52D4C89B02378BC
:102E8000002B4FD1FEF73EFD02232A4F03903A68F4
:102E90001A42FCD120230693069B5A1E0692002B51
:102EA000FAD1254E3368002BFCDA0120FFF7A2FF90
:102EB000011E02D0112009B0F0BD030003220190D1
:102EC000009005AD9F2000F037FD0321280000F0A1
:102ED000FBFD02233A681A42FCD120230793079B8B
:102EE0005A1E0792002BFAD13368002BFCDA01201E
:102EF000FFF780FF0028DDD10398FEF717FDAA78C1
:102F00006B7811041B020B4329780B436360130099
:102F1000113B0A49052B07D801239340A3600B609E
:102F2000012323700020C6E780231B03F6E7C04679
:102F3000BC3DFF1F90C8004000C800409808FF1F1C
:102F40001E4B30B55A6818781D4B85B0D3185942BE
:102F50004B4101210093002300F096FB194B1A4AC4
:102F600002259A6300221A6510325A658022C42114
:102F70009D65164B1648D202DA6789004258154BF8
:102F800080241A4080231B041343435064234120B0
:102F90000393E40500F006FA402000F003FA6562AE
:102FA000039D6B1E0393002DFAD103236362FFF789
:102FB0003BFFA562FFF760FF05B030BDC83DFF1FB6
:102FC00095FFFEF700C80040050001FF04E100E0A6
:102FD00000E100E0FFFF00FFF0B585B00700FEF75D
:102FE00091FC022305002D4C22681A42FCD12023BB
:102FF0000093009B5A1E0092002BFAD1284E336892
:10300000002BFCDA0120FFF7F5FE002803D0112485
:10301000200005B0F0BD234B2360022322681A4232
:10302000FCD120230193019B5A1E0192002BFAD15F
:103030003368002BFCDA0120FFF7DCFE0028E6D124
:10304000194B1F60022322681A42FCD120230293ED
:10305000029B5A1E0292002BFAD13368002BFCDA35
:103060000120FFF7C7FE0028D1D1104B23600223B7
:1030700022681A42FCD120230393039B5A1E039219
:10308000002BFAD13368002BFCDA0120FFF7B2FEE7
:10309000041EBCD12800FEF749FCB9E790C80040E7
:1030A00000C8004001000006A8C8004001800001DF
:1030B00010B50020FFF790FF10BD000010B5064BC3
:1030C00018705960FFF73CFF00211320034AFFF7F7
:1030D00057FD002010BDC046C83DFF1F412FFF1FF8
:1030E000F0B5040085B003920291FEF70BFC882234
:1030F00063035B0B52051A438023DB059D6A802323
:10310000274F0092BA68002601901B039A420CD9FF
:10311000F82326001B041E401C4206D08022214BAF
:1031200052025E6219680A431A60002D0BD100F04A
:10313000DBFB02221C4B1A608023DB055A62013A3A
:103140009A6200F079FC0023039A934220D1002D6B
:103150000AD100F0C9FB144B03221D608023DB055C
:103160005A629D6200F068FC8023BA681B039A4291
:1031700008D9002E06D000220A4B0C495A621A6860
:103180000A401A600198FEF7D1FB002005B0F0BD9F
:10319000009A0299D2181278CA540133D4E7C04673
:1031A000BC3DFF1F00C8004000C00040FFFFFEFF05
:1031B000F0B587B0029103920400FEF7A3FB0190E3
:1031C00000F092FB802302250122234EDB053560AF
:1031D0005D629A6200F030FC204F3B682B42FCD1CC
:1031E00020230493049B5A1E0492002BFAD11C4DF9
:1031F0002B68002BFCDA0120FFF7FCFD002802D031
:10320000112007B0F0BD2000039A029900F0ACFA3B
:10321000022304003A681A42FCD120230593059B3F
:103220005A1E0592002BFAD12B68002BFCDA0120E4
:10323000FFF7E0FD051EE3D100F056FB80230322DB
:10324000DB0535605A629D6200F0F6FB0198FEF7DF
:103250006DFBE0B2D5E7C04600C0004090C800401A
:1032600000C80040F0B5802489B00600FEF74AFB94
:10327000E405A36A02250393029000F035FB0123C5
:10328000304F3D606562A36200F0D6FB2E4C236890
:103290002B42FCD120230593059B5A1E0592002B3F
:1032A000FAD12A4D2B68002BFCDA0120FFF7A2FD92
:1032B000002803D01124200009B0F0BD244B236066
:1032C000022322681A42FCD120230693069B5A1E31
:1032D0000692002BFAD12B68002BFCDA0120FFF7B5
:1032E00089FD021EE6D11B4B03211E6003000190E5
:1032F0000090202000F020FB022322681A42FCD11B
:1033000020230793079B5A1E0792002BFAD12B68A4
:10331000002BFCDA0320FFF76DFD041ECAD100F07C
:10332000E3FA80230322DB053C605A629C6200F0D2
:1033300083FB039B002B01D1FFF776FD0298FEF77C
:10334000F5FAB8E700C0004090C8004000C800404F
:103350000100000694C8004007B500020191042254
:10336000000A01A9FFF724FF0EBD000073B5050098
:1033700005240B4AA3005B429B1819686B46DE1DAF
:103380003000FFF7B3FA022804D133782B55013C03
:10339000EFD276BD052CFCD00128FAD10230F8E737
:1033A000140900111F2807D8012380228340D20569
:1033B00091680B43936070473F2808D8012380220F
:1033C00020388340D20551690B435361F3E75F28EE
:1033D000F1D80123802240388340D205116A0B4383
:1033E0001362E8E71F2807D8012280218240C9051F
:1033F0008B6893438B6070473F2808D80122802157
:1034000020388240C9054B6993434B61F3E75F283D
:10341000F1D80122802140388240C9050B6A9343CC
:103420000B62E8E71F2810D880230200DB05153A5D
:103430001968012A06D820229143196019680A43A5
:103440001A60704701228240F6E73F2811D8802396
:103450000200DB05353AD968032A06D810229143C9
:10346000D960D9680A43DA60EBE70122203882404C
:10347000F5E75F28E5D842238022181A413B8340B4
:10348000D205516A99435162516A0B435362D8E79E
:1034900010B50400012813D1A022184992050B6829
:1034A0005B015B0913430B60154B164A1968114009
:1034B000154A0A431A60402219680A431A6010BD6F
:1034C0000028FCD101000A2000F056F921000B2051
:1034D00000F052F9C0220A4B920019680A434021B9
:1034E0001A601A688A431A60B022044912060B68EF
:1034F0005B015B0913430B60E1E7C04614F0004039
:103500001CF000407F00FEFF80FD010072B6074AFC
:103510001368013313600422054B1A600023054A27
:1035200013608022D2055360FEE7C0467808FF1F73
:10353000C0F00040C4F0004005490B68002B05D1E5
:10354000044A0A6004490A60044A13607047C0468E
:10355000140AFF1F841E0000380AFF1FC4F0004039
:103560000023034A1360034A1360034A1360704741
:1035700054F0004040F1004044F10040002310B5F9
:10358000184C8AB0009301932378012B27D0694609
:10359000012000F011F9002817D1009B1249029375
:1035A000019B06AA0393114B02A81B680493104BBE
:1035B0001B68059300F0E8F910220E4906A800F0F8
:1035C00093F8002804D1FF23237000200AB010BD17
:1035D0000123094A074902A8237000F0D5F9012008
:1035E000F4E7C046B05EFF1F102900110829001142
:1035F0000C29001120290011B45EFF1F13B501240E
:103600006946012000F0D8F8034B00940193FFF7BE
:10361000B5FF200016BDC046BB0B000010B5FFF77C
:103620009FFFFFF7EBFF002802D0024B984710BD29
:10363000FEE7C046E1A2000002B471464908490015
:10364000095649008E4402BC7047C04602B4714618
:1036500049084900095C49008E4402BC7047C046D5
:1036600003B47146490840004900095A49008E4494
:1036700003BC70470000000001B40248844601BC4E
:10368000604700BFDD0C010001B40248844601BC64
:10369000604700BFC56D010001B40248844601BC0B
:1036A000604700BFBD5C010001B40248844601BC14
:1036B000604700BF7997000001B40248844601BC0E
:1036C000604700BF5976010001B40248844601BC3E
:1036D000604700BF53B9000001B40248844601BCF2
:1036E000604700BFE917010001B40248844601BCED
:1036F000604700BFCD4C010001B40248844601BCC4
:10370000604700BF116E000001B40248844601BC4E
:10371000604700BF6DF6000001B40248844601BC5A
:10372000604700BF8D11010001B40248844601BC0E
:10373000604700BFC1F7000001B40248844601BCE5
:10374000604700BF71B0000001B40248844601BC6C
:10375000604700BF8914010001B40248844601BCDF
:10376000604700BF8512010001B40248844601BCD5
:10377000604700BF9573010001B40248844601BC54
:10378000604700BFFDA1001101B40248844601BC9E
:10379000604700BF156B010001B40248844601BCBC
:1037A000604700BF7912010001B40248844601BCA1
:1037B000604700BF2D6C010001B40248844601BC83
:1037C000604700BFE1AC000001B40248844601BC80
:1037D000604700BF51B8000001B40248844601BCF4
:1037E000604700BF8552010001B40248844601BC15
:1037F000604700BFED6B010001B40248844601BC84
:10380000604700BF0534010001B40248844601BC92
:10381000604700BF8944000001B40248844601BCEF
:10382000604700BF6911010001B40248844601BC31
:10383000604700BFE512010001B40248844601BCA4
:10384000604700BFF535010001B40248844601BC61
:10385000604700BFD1AE000001B40248844601BCFD
:10386000604700BFDD0A010001B40248844601BC84
:10387000604700BFC9A9000001B40248844601BCEA
:10388000604700BFE94C010001B40248844601BC16
:10389000604700BFF90D010001B40248844601BC35
:1038A000604700BF8D82000001B40248844601BC1D
:1038B000604700BFED68010001B40248844601BCC6
:1038C000604700BFB70E000001B40248844601BC47
:1038D000604700BF6137010001B40248844601BC63
:1038E000604700BFC95C010001B40248844601BCC6
:1038F000604700BF75A9000001B40248844601BCBE
:10390000604700BF2144000001B40248844601BC66
:10391000604700BF090E000001B40248844601BCA4
:10392000604700BF4DF9000001B40248844601BC65
:10393000604700BFE927000001B40248844601BC8B
:10394000604700BF496D010001B40248844601BCD4
:10395000604700BFC115010001B40248844601BCA4
:10396000604700BFADAE000001B40248844601BC10
:10397000604700BF0934010001B40248844601BC1D
:10398000604700BF79B5001101B40248844601BC0C
:10399000604700BFDD3F000001B40248844601BC1F
:1039A000604700BFC166010001B40248844601BC03
:1039B000604700BFE90B010001B40248844601BC26
:1039C000604700BF090E000001B40248844601BCF4
:1039D000604700BF0189000001B40248844601BC71
:1039E000604700BFD544010001B40248844601BCD1
:1039F000604700BF21A9000001B40248844601BC11
:103A0000604700BFEDA5000001B40248844601BC38
:103A1000604700BF6D0B010001B40248844601BC41
:103A2000604700BF01D7000001B40248844601BCD2
:103A3000604700BF85C1000001B40248844601BC54
:103A4000604700BF9DA9000001B40248844601BC44
:103A5000604700BFBD0B010001B40248844601BCB1
:103A6000604700BFCD0C010001B40248844601BC90
:103A7000604700BFE9D4000001B40248844601BC9D
:103A8000604700BF0134010001B40248844601BC14
:103A9000604700BF016C010001B40248844601BCCC
:103AA000604700BF0167010001B40248844601BCC1
:103AB000604700BFD9B0000001B40248844601BC91
:103AC000604700BFF935010001B40248844601BCDB
:083AD000604700BF3D710100D9
:103AD800020000000EBE00110100000020BC001111
:103AE800020000000ABE001101000000183BFF1F81
:103AF8000200000028BC001101000000285CFF1F24
:103B08000200000008BE0011030000009C5BFF1FBC
:103B180012000000020000000EBE001101000000AB
:103B280068BC0011020000000ABE0011010000007C
:103B380065BC00110200000072BC00110300000007
:103B4800D75BFF1F0200000008BE00110300000041
:103B5800EC5BFF1F020000000ABE0011010000001C
:103B680064BC00110200000070BC001103000000DA
:103B7800AD5BFF1F0200000008BE0011030000003B
:103B8800CE5BFF1F020000000EBE00110100000006
:103B9800A8BC0011020000000ABE001101000000CC
:103BA800613CFF1F02000000BABC001101000000C8
:103BB800A3BC0011020000000ABE001101000000B1
:103BC800603CFF1F02000000B8BC001101000000AB
:103BD800F45BFF1F020000000ABE00110100000094
:103BE8005F3CFF1F02000000B6BC0011010000008E
:103BF80093BC0011020000000ABE00110100000081
:103C08005E3CFF1F02000000B4BC00110100000070
:103C18008EBC0011020000000ABE00110100000065
:103C28005D3CFF1F02000000B2BC00110100000053
:103C380089BC0011020000000ABE0011010000004A
:103C48005C3CFF1F02000000B0BC00110100000036
:103C580084BC0011020202020202000000000000FF
:103C680016150000954B00115B4B0011FCBC0011B0
:103C780090011D0018001800FFFF0701020304054A
:103C8800060201060000000000000000000000001D
:103C9800000000000000000000000000000000001C
:103CA80003000000020000000EBE00110100000029
:103CB8001CBD0011020000000ABE00110100000036
:103CC8001C3DFF1F0200000026BD0011010000007E
:103CD800225CFF1F0200000008BE00110300000064
:103CE8008C5EFF1F020000000ABE001101000000E8
:103CF8001C3DFF1F0200000024BD00110100000050
:103D0800245CFF1F0200000008BE00110300000031
:103D1800845EFF1F12A6A6A6000000000000000097
:103D2800161500000001000000000111FFFF00004F
:103D38005048593600000000000000000B00050044
:103D4800F0000000B4000028002800283075A0000A
:103D5800A000A000A00000080008E001F00010008A
:103D6800100010001000100010005000500050000B
:103D780010001000D0070000000000000F00010034
:103D88000500307507001000010081FF00000000E9
:103D9800FF000000E5730011ED7100117D6F001147
:103DA800FFFF0100FF000000019E00117D9B001134
:103DB800959A0011000000000000000000000800B3
:103DC800040000003B0001085902E0018821280096
:103DD800020000000EBE001101000000D4BE001158
:103DE800020000000ABE001101000000553EFF1F3E
:103DF8000200000006BE0011010000006C62FF1FF7
:103E0800020000000ABE001101000000543EFF1F1E
:103E18000200000004BE001101000000523EFF1F16
:103E2800020000000ABE001101000000503EFF1F02
:103E38000200000002BE001101000000483EFF1F02
:103E4800180018001D009001020000030202000083
:103E5800020000000EBE001101000000E8BE0011C3
:103E6800020000000ABE001101000000983EFF1F7A
:103E78000200000000BE0011000000000000000069
:103E88000200000008BE0011030000008C62FF1F42
:023E980020FF09
:040000051FFF184180
:00000001FF
